:020000040800F2
:10000000480D002075C8000871C5000873C50008B8
:1000100075C5000877C5000879C500080000000014
:100020000000000000000000000000007BC5000888
:100030007DC50008000000007FC5000881C50008DC
:10004000ADC8000883C50008B1C80008B5C80008DD
:10005000B9C80008BDC80008C1C80008C5C8000864
:10006000C9C80008CDC80008D1C80008D5C8000814
:10007000D9C80008DDC80008E1C80008E5C80008C4
:10008000E9C80008EDC80008F1C80008F5C8000874
:10009000F9C80008FDC8000801C9000887C50008A4
:1000A00005C900088DC5000809C900080DC9000868
:1000B00011C9000815C9000819C900081DC90008A0
:1000C00021C9000825C9000829C9000893C50008EE
:1000D0002DC9000831C9000835C9000839C9000810
:1000E0003DC9000841C9000845C9000849C90008C0
:1000F0004DC9000851C9000855C9000859C9000870
:100100005DC9000861C9000865C9000869C900081F
:1001100099C500089FC500086DC9000871C900088D
:1001200075C9000879C900087DC9000881C900089F
:1001300085C9000889C900088DC9000891C900084F
:1001400095C9000899C900089DC90008A1C90008FF
:10015000A5C90008A9C90008ADC90008B1C90008AF
:10016000B5C90008B9C90008BDC90008C1C900085F
:10017000C5C90008C9C90008CDC9000800000000B1
:10018000D1C90008D5C90008D9C90008DDC90008CF
:10019000E1C90008E5C90008E9C90008EDC900087F
:1001A000F1C90008F5C90008F9C90008FDC900082F
:1001B00001CA000800F5E0700268914203D3436869
:1001C0001A44914202D380680028F5D1704718493B
:1001D000086880B94FF4805048604FF480324FF087
:1001E000FF30C86008610420124B8A604861C3F880
:1001F000BC01114808600120704701F1080313F0A9
:10020000070F0EBF0023C3F1080303F007031944CF
:10021000D21A8161C26042F001034B60091D4FF0A8
:10022000280C41F802C0024A1369C36170470000FC
:1002300018090020E00500206859883C2DE9F84F96
:1002400084B00646AFF30080F52E1E4D80F0138279
:100250000B2E31BF10260B36F608F6002868F4087E
:10026000E04010F0030F4AD0C04300F00100041931
:1002700005F1280000EBC408E700D8F808607068B2
:10028000C008C000B84218BF01F016FAD6F80890AE
:10029000464508BF01F010FA4E4508BF01F00CFAC0
:1002A0007068C008C000B84218BF01F005FAC84520
:1002B0000AD12868012101FA04F420EA04042C6020
:1002C00010E000BFE00500202869814508D3D9F877
:1002D0000C10B14204D1C8F80890C9F80C8001E0B4
:1002E00001F0EAF947F00300311D7060301DCA5972
:1002F00042F00102C25106F1080800F01DBFA968D2
:10030000B14280F0A883002800F0A2804FF00108DD
:1003100008FA04F1490000FA04F4484201430C4091
:1003200060420440641E200B00F01000C4406109CC
:1003300001F00801CC40A20802F00402D440630896
:1003400003F002030818DC401018C4F34007181823
:100350003818FC40241805F1280000EBC40AE70017
:10036000DAF80890D9F80400C008C000B84218BFF5
:1003700001F0A2F9D9F808B0D14508BF01F09CF905
:10038000D94508BF01F098F9D9F80400C008C000A9
:10039000B84218BF01F090F9DA4506D1286808FA8A
:1003A00004F420EA04042C600DE029698B4508D38D
:1003B000DBF80C00484504D1CAF808B0CBF80CA013
:1003C00001E001F079F9BF1B46F0030009F10402D6
:1003D000C9F8040047F00101915109EB06020192AE
:1003E000D751AC684FEAD40ABAF11F0F88BF01F0A9
:1003F00063F934B3CDF800A005F128006E6900EB75
:10040000CA0AD346102C38BF01F056F92968009863
:1004100021FA00F2D30704D408FA00F00843286058
:1004200007E0DAF80800296988422CBF834601F00A
:1004300043F9CAF80860CBF80C60C6F808B0C6F8F3
:100440000CA0AF6009F108080198686100F074BE63
:100450006868002800F0208341420840401E010BDC
:1004600001F01001C840420902F00802D0408308A0
:1004700003F00403D840440804F002045118E0409B
:100480005918C0F34007611805F598787918F840B5
:10049000401858F820104868C008C0008A46A0EBF1
:1004A000060B08E001464868C008C000801B58459C
:1004B0003CBF83468A4608690028F3D14969002970
:1004C000F1D128698245C0F0D380DAF80410C90858
:1004D00006EB0B09C900494518BF01F0EDF80AEB1E
:1004E00006008245019080F0C380DAF80C40DAF80B
:1004F000187054450DD0DAF808002969884223D3D2
:10050000C268524504BFA16851451DD1C460A060B6
:100510001CE00AF114010C6834B90AF110010C68EE
:10052000A4B101E011460C6804F11402106800281F
:1005300002BF04F1100210680028F3D1286981423B
:1005400002D300220A6001E001F0B6F8002F38D093
:10055000DAF81C0008EB80010A6892450AD11CBB3E
:100560006A68012303FA00F022EA000068600020B4
:10057000086026E029698F4213D33869504514BFBB
:100580007C613C61ECB129698C4218D3A761DAF82F
:10059000100058B1884226BF2061846101F08CF8B8
:1005A00004E001F089F8EDE70C60ECE7DAF81400FC
:1005B00038B12969884202D36061846101E001F0A9
:1005C0007BF8BBF1100F0ED249F003000AF10401D1
:1005D000CAF804000AF1040051F8092042F00102AF
:1005E00040F809203EE046F003010AF10402CAF88F
:1005F00004104BF001009051019941F80BB0A8682C
:100600000090C4081F2C88BF01F056F8009828B34A
:1006100005F1280000996F6900EBC408C146102954
:1006200038BF01F049F8286820FA04F1CA0705D458
:10063000012101FA04F404432C6007E0D8F8080013
:10064000296988422CBF814601F036F8C8F8087045
:10065000C9F80C70C7F80890C7F80C80C5F808B046
:10066000019868611AF1080800F0F58100F064BD96
:1006700001F022F8EFE116F1400F28BF4FF0FF36EE
:1006800080F0E9810B36F6086B68F600002B00F06D
:10069000E2810027300AC6F1000908BF002423D0F8
:1006A000B0F5803F28BF1F241ED2A0F58071090C31
:1006B00001F008018840A0F58052120C02F00402FB
:1006C0009040A0F58044240CC1F10E0104F0020416
:1006D000891A091BA04001EBD031C81D26FA00F48D
:1006E00004F0010404EB410405F5987858F824005F
:1006F00030B31F2C0FBFB4464FEA540CCCF1190C89
:1007000006FA0CFCBE46494601E04FEA4C0C426832
:10071000D208D200921B8A4202D2110007460CD0A6
:10072000426910304FEADC7950F82900002A1CBFDA
:10073000824296460028E8D170468946A8BBB7BBDE
:10074000012101FA04F4640060420443234000F0F4
:100750008281584203405B1E180B00F01000C3401A
:10076000590901F00801CB409A0802F00402D34075
:100770005C0804F002040818E3401018C3F3400CAE
:100780002018604423FA0CF31B1858F823000CE0DF
:1007900008464168C908C900891B49453CBF8946CC
:1007A000074601690029F3D140690028F1D1002FE3
:1007B00000F05181A868801B814580F04C81296937
:1007C0008F42FFF455AF7868C008C00006EB0901FE
:1007D000884218BF00F070FF07EB060B5F45BFF4BF
:1007E00047AFFC68D7F818A0BC420CD0B86829699C
:1007F000884223D3C268BA4204BFA168B9421DD15E
:10080000C460A0601CE007F114010C6834B907F162
:1008100010010C68A4B101E011460C6804F1140247
:100820001068002802BF04F1100210680028F3D1FC
:100830002869814202D300220A6001E000F03CFFF7
:10084000BAF1000F39D0F86908EB80010A689742C5
:100850000AD134BB6A68012303FA00F022EA0000DF
:1008600068600020086028E029698A4516D3DAF814
:100870001000B84214BFCAF81440CAF81040E4B1DE
:1008800029698C4217D3C4F818A0386958B1884236
:1008900026BF2061846100F00FFF04E000F00CFF30
:1008A000EDE70C60ECE7786938B12969884202D33A
:1008B0006061846101E000F0FFFEB9F1100F0CD21D
:1008C000B14449F00300391D7860381D51F8092002
:1008D00042F0010240F80920B9E046F003013A1D58
:1008E000796049F0010090514FEAD9004BF8099026
:1008F0001F2822D805F1280101EBC004296821FA3C
:1009000000F2D307A04605D4012202FA00F0084302
:10091000286006E0A068296988422CBF804600F064
:10092000CBFEC4F808B007F10800C8F80CB040F8D6
:10093000068007F10C018C5189E05FEA192008BF9D
:10094000002123D0B0F5803F28BF1F211ED2A0F583
:100950008072120C02F008029040A0F58051090C40
:1009600001F004018840A0F580431B0CC2F10E0287
:1009700003F00203521AD21A984002EBD032D01D73
:1009800029FA00F101F0010101EB420107F1140322
:10099000CBF81C1000229A5107F1100308EB8100DC
:1009A0009A516A6822FA01F3DC0711D4012303FA91
:1009B00001F111436960C0F800B0CBF8180007F1ED
:1009C000080107F10C0040F806B041F806B03EE01F
:1009D00002681F291DBF4908C1F1190109FA01F177
:1009E000494600E002465068C008C000484518D09B
:1009F00002F11003C80F03EB8003490018680028B8
:100A0000F0D12869834220D3C3F800B007F10C016C
:100A1000CBF8182041F806B007F1080040F806B0FE
:100A200015E0296990688A4228BF88420DD3C0F832
:100A30000CB007F10801C2F808B0885107F10C00AA
:100A400082510022CBF8182001E000F035FE17F1AA
:100A5000080840F07183A868B0421DD3811B6A6901
:100A6000102909D39319A96041F001005860595029
:100A700046F0030656600BE00021A96040F0030435
:100A8000111D5460141D0E5846F001062650002317
:100A90006B6102F108084FE3E8688642C0F03C83CE
:100AA000DFF8CC9BD9F8000008B9FFF790FBD9F824
:100AB000081088192F30491E20EA01018E4280F06B
:100AC000398305F5D877B86838B13A6889188A4209
:100AD00080F030838842C0F02D8300F00DFE0028A6
:100AE0001CBFD0F8008010F1010F00F0238339689B
:100AF0007A68414439608A4238BF7960AC6904BB86
:100B0000296909B1884200D2286100213861C7F8FB
:100B10001480F9614FF0FF31D9F800206A62296230
:100B200005F1280200219260D26002F108035361AE
:100B30001361891C10321F29F5D9A8F1280201463A
:100B40001DE005F5E0710A46814600E09268D2B1E9
:100B50001068536803449945F8D1107B030712D4F9
:100B600013689C420FD3D2F804C063449C420AD25B
:100B7000C444C2F804C02146E86808EB00022846D5
:100B8000FFF73BFBC5E22869814538BFC5F81090E7
:100B900009EB080000E08968002900F0C1810A68BB
:100BA0008242F8D1087B020700F1BA810868C1F8D7
:100BB00000904A6842444A6009F1080111F0070FA9
:100BC00008BFCDF8049006D0C1F1080101F007017B
:100BD00009EB0102019200F1080111F0070F04D0A6
:100BE000C1F1080101F00701084480460198A8EB13
:100BF00000018419A1EB060B274646F00306466068
:100C0000474528BF00F058FD98F80400C10758BFB9
:100C100000F052FDBBF1100F38BF00F04DFDA86988
:100C2000804508D1E9688B44C5F80CB0AF614BF042
:100C30000100786070E1686980450AD1A9686F6138
:100C40008B44C5F808B04BF00100786047F80BB052
:100C500062E1D8F8040000F00301012940F0BC80F3
:100C6000C008C000C1081F29039040D8D8F8082048
:100C70000092D8F80C600291B04508BF00F01CFD4E
:100C80000098804508BF00F017FDD8F804000299CD
:100C9000C008C000B0EBC10F18BF00F00DFD0299F5
:100CA000009A05F1280000EBC100824208D01146ED
:100CB0002A699142C0F08B80CA68424540F0878023
:100CC00000998E4206D102982A68012383409A43F4
:100CD0002A607EE0864205D029698E4277D3B068CB
:100CE000404574D10098C6600099B16071E0D8F8B1
:100CF00018000090D8F80C6046450DD0D8F80800D0
:100D00002969884223D3C268424504BFB16841457E
:100D10001DD1C660B0601CE008F114010E6836B940
:100D200008F110010E68A6B101E011460E6806F147
:100D300014021068002802BF06F110021068002893
:100D4000F3D12869814202D300220A6001E000F059
:100D5000B3FC009800283CD0D8F81C0005F5987129
:100D600001EB80010A6890450AD12EBB6A68012315
:100D700003FA00F022EA000068600020086028E022
:100D800000992869814214D30869404514BF4E6117
:100D90000E61F6B129698E4219D30098B061D8F876
:100DA000100058B1884226BF3061866100F084FC93
:100DB00004E000F081FCECE70E60EBE7D8F81400EB
:100DC00038B12969884202D37061866101E000F080
:100DD00073FC039988448B44D8F8041049084900EF
:100DE000C8F804104BF0010078604FEADB0647F8C2
:100DF0000BB01F2E22D805F1280000EBC604A14637
:100E0000BBF1100F38BF00F057FC286820FA06F13C
:100E1000CA0705D4012101FA06F606432E6006E052
:100E2000A068296988422CBF814600F045FCA76074
:100E3000C9F80C70C7F80890FC606DE05FEA1B20F1
:100E400008BF002123D0B0F5803F28BF1F211ED24C
:100E5000A0F58072120C02F008029040A0F58051BB
:100E6000090C01F004018840A0F580431B0CC2F17D
:100E70000E0203F00203521AD21A984002EBD0324B
:100E8000D01D2BFA00F101F0010101EB4201F961E3
:100E9000002305F598727B6102EB81003B616A6873
:100EA00022FA01F3DE0707D4012303FA01F111430B
:100EB00069600760B8611DE002681F291DBF49080D
:100EC000C1F119010BFA01F1594600E002465068E0
:100ED000C008C000584510D002F11003C80F03EB42
:100EE0008003490018680028F0D12869834211D393
:100EF0001F60BA61FF60BC600EE0296990688A4299
:100F000028BF884206D3C7609760B860FA600020A7
:100F1000B86101E000F0D0FB019800F108080BE196
:100F200021462846FFF746F90168406808440090CA
:100F3000A0F1270111F0070000980EBF0021C1F1B8
:100F4000080101F007010844A0F12F0B04F1100182
:100F50008B4538BFA3460BF1180200210292019184
:100F6000A8F1280249462846FFF747F90BF1080087
:100F700010F0070F18BF00F09FFB1B20CBF80400F8
:100F800005F5E07292E809500BF1080181E809507B
:100F900000210BF10800F961B861009A02980199EB
:100FA000C7F81090C7F81480072300E0001D491C03
:100FB00000F1080797424360F8D30129D8BF00F039
:100FC0007BFBA34500F0A580ABEB040B201D221D8D
:100FD00050F80B104908490042F80B104BF0010083
:100FE00060604FEADB0944F80BB0B9F11F0F22D85B
:100FF00005F1280000EBC907B846BBF1100F38BF58
:1010000000F05AFB286820FA09F1CA0705D401212B
:1010100001FA09F10843286006E0B86829698842A6
:101020002CBF804600F048FBBC60C8F80C40C4F8F8
:101030000880E7606DE05FEA1B2008BF002123D035
:10104000B0F5803F28BF1F211ED2A0F58072120C80
:1010500002F008029040A0F58051090C01F0040153
:101060008840A0F580431B0CC2F10E0203F002037E
:10107000521AD21A984002EBD032D01D2BFA00F14E
:1010800001F0010101EB420105F59872002302EB2A
:101090008100E161636123616A6822FA01F3DF077D
:1010A00007D4012303FA01F1114369600460A061D0
:1010B0001DE002681F291DBF4908C1F119010BFA83
:1010C00001F1594600E002465068C008C00058458A
:1010D00010D002F11003C80F03EB80034900186819
:1010E0000028F0D12869834211D31C60A261E4601A
:1010F000A4600EE0296990688A4228BF884206D31E
:10110000C4609460A060E2600020A06101E000F093
:10111000D3FAE86886420DD2801BA969E8608A1973
:10112000AA6140F00100506046F003064E6001F1F4
:10113000080801E04FF00008AFF30080404605B01A
:10114000BDE8F08F002800D170472DE9F047A0F1ED
:101150000805AFF30080DFF85C6531698D42C0F0AF
:101160008482686800F00302012A00F07E82C208CF
:101170004FEAC209C20705EB090839D42C6810F000
:10118000030F00F06E82604205448D42A144C0F01E
:101190006C827069854200F0DE80E408202C72D2F7
:1011A000D5F80CA0AF68554508BF00F085FABD42E0
:1011B00008BF00F081FA6868C008C000B0EBC40F37
:1011C00018BF00F079FA06F1280000EBC40087424E
:1011D00005D031698F4253D3FA68AA4250D1BA453B
:1011E00040D13068012101FA04F420EA040434609B
:1011F000454580F03A82D8F80440E00740F1358256
:10120000A10700F18381B069804540F0B780F168A3
:10121000B5618944C6F80C9049F0010068607169B5
:101220008D4202D100207061B060F169494580F0C3
:101230001882DFF83C24106808B9FEF7C8FFB169CE
:10124000002900F00E82F068292824BF3046FEF7FE
:10125000B1FFF069F168884280F003824FF0FF30FF
:10126000F061FEE1824506D03069824508D3DAF8A4
:101270000810A94204D1C7F80CA0CAF80870B7E753
:1012800000F01AFAB4E7EC68AF69AC420BD0A8687A
:10129000884222D3C168A94204BFA268AA421CD1D5
:1012A000C460A0601BE005F11402146834B905F1B4
:1012B000100214689CB101E01A46146804F114038A
:1012C0001868002802BF04F1100318680028F3D141
:1012D0008A4202D30021116001E000F0EDF9002FF5
:1012E00086D0E86906F5987101EB80010A6895429D
:1012F0000AD124BB7268012303FA00F022EA00003D
:1013000070600020086073E731698F4214D3386938
:10131000A84214BF7C613C61002C3FF469AF316985
:101320008C42ADD3A761286958B1884226BF20619D
:10133000846100F0C1F904E000F0BEF9ECE70C6054
:10134000EDE7686900283FF453AF3169884297D3CD
:10135000606184614CE798F8040000F00300032802
:101360007FF446AFC6F8089049F00101D8F80400B0
:1013700040084000C8F8040069600AE070698045D0
:101380000AD1B16875618944C6F8089049F0010036
:10139000686045F8099064E1E408E400A144E408C9
:1013A000202C3AD2D8F80CA0D8F80870D04508BF45
:1013B00000F082F9B84508BF00F07EF9D8F80400C3
:1013C000C008C000B0EBC40F18BF00F075F906F1FB
:1013D000280000EBC400874207D031698F42C0F07B
:1013E0008880FA68424540F08480BA4507D1306869
:1013F000012101FA04F420EA040434607BE0824510
:1014000006D03069824574D3DAF80810414570D1AE
:10141000C7F80CA0CAF808706DE0D8F80C40D8F8EE
:10142000187044450DD0D8F808003169884223D39C
:10143000C268424504BFA16841451DD1C460A06097
:101440001CE008F114010C6834B908F110010C68B3
:10145000A4B101E011460C6804F1140210680028E0
:1014600002BF04F1100210680028F3D130698142F4
:1014700002D300220A6001E000F01EF9002F3AD0EA
:10148000D8F81C0006F5987101EB80010A689045B8
:101490000AD11CBB7268012303FA00F022EA0000A3
:1014A00070600020086026E031698F4213D33869EC
:1014B000404514BF7C613C61ECB131698C4218D36A
:1014C000A761D8F8100058B1884226BF2061846116
:1014D00000F0F2F804E000F0EFF8EDE70C60ECE764
:1014E000D8F8140038B13169884202D36061846150
:1014F00001E000F0E1F849F00100686045F809906A
:1015000071698D420BD1C6F80890AAE064086400A6
:10151000C8F8044049F00100686045F809904FEAB6
:10152000D907202F22D206F1280000EBC704A046DD
:10153000B9F1100F38BF00F0BFF8306820FA07F19A
:10154000CA0705D4012101FA07F70743376006E00F
:10155000A068316988422CBF804600F0ADF8A560D4
:10156000C8F80C50C5F80880EC607AE05FEA1920F2
:1015700008BF002123D0B0F5803F28BF1F211ED215
:10158000A0F58072120C02F008029040A0F5805184
:10159000090C01F004018840A0F580431B0CC2F146
:1015A0000E0203F00203521AD21A984002EBD03214
:1015B000D01D29FA00F101F0010101EB420106F50D
:1015C0009872002302EB8100E9616B612B61726804
:1015D00022FA01F3DC0707D4012303FA01F11143D6
:1015E00071600560A8611DE002681F291DBF4908E0
:1015F000C1F1190109FA01F1494600E002465068BB
:10160000C008C000484510D002F11003C80F03EB1A
:101610008003490018680028F0D13069834211D353
:101620001D60AA61ED60AD600EE0316990688A428C
:1016300028BF884206D3C5609560A860EA60002094
:10164000A86101E000F038F8306A401E08D130622D
:10165000D6F8C80100E080680028FCD14FF0FF30C8
:101660003062AFF30080BDE8F08700F025F8F8E7BE
:101670001809002038B5002558B141EA0002120CC3
:1016800001FB00F512041EBFB5FBF0F088424FF0DD
:10169000FF352846FEF7D2FD04001CBF14F8040CE9
:1016A00010F0030F03D02946204600F03BF82046F7
:1016B00032BD0000E0050020012000F049B830B440
:1016C000002513E050F8042BD30744BFA9F1010310
:1016D0009A18091F042942F8045BFAD213468C07B2
:1016E00044BF15809B1CC90748BF1D7050F8041BE0
:1016F0000029E7D130BC70470749086808B10020CD
:1017000070470648C008C00008600549C908C900FC
:10171000091A0160704700BF3C0900204F0D0020EE
:10172000480F0020002200F021B8B1F5807F02D3DD
:101730004FF0FF3070470170012070470A78026057
:10174000087800E00078401E8041C043C00F704719
:1017500080B500F03BF8024A11001820ABBEFBE751
:101760002600020062F30F2262F31F42401810F0BD
:10177000030308D0C91A1FD3DB0748BF00F8012DA7
:1017800028BF20F8022D130030B414461546103936
:1017900028BF20E93C00FAD8490728BF20E90C00FF
:1017A00048BF40F8042D890028BF20F8022D48BF0B
:1017B00000F8012D30BC7047C91818BF00F8012D82
:1017C000CB0728BF00F8012D70472E0010B500F0A0
:1017D00052F8020000230024E4431068A04203D022
:1017E00011000220ABBE13605068A04203D0111D4F
:1017F0000220ABBE536010BDF0B583B0040000F012
:101800003AF8A10047183D680026F643B54216D1C4
:1018100000F01AF83D68B5420FD100BF09A0009052
:10182000002C01D1002000E0042001900320029050
:1018300069460120ABBE05003D6000F014F82800A9
:1018400003B0F0BD3A7474000C480121BFF35F8F00
:10185000D0E84F3FC0E8421F002AF9D1BFF35F8FA5
:10186000002BF3D170470548BFF35F8F0021017053
:10187000BFF35F8F704702487047000040090020A7
:10188000F80200202DE9FE4F5FF0000632A40FF2AF
:1018900048390FF24C3A0FF2D40BDFF8788D00F094
:1018A00003F91F462DE000F04DFB29E0002FFAD18F
:1018B000584601F051FA00F0A5F9717800F0A3F94B
:1018C000B17800F0A0F9F17800F09DF9317900F0DD
:1018D0009AF9717900F052FA00F03FFCB17B00F008
:1018E00092F9F17B00F08FF9317C00F08CF9717C7A
:1018F00000F089F9B17C00F086F9F17C00F03EFA45
:101900002E469DF80100864223DA00F02AFF9DF85A
:1019100000000428F4D100F071F94E438119012F21
:1019200001F1A20612D1584601F016FA00F06AF948
:10193000717800F068F9B17800F065F9F17800F09D
:1019400062F9317900F05FF97179D7E7022FADD1F3
:10195000C2E7BDE8F78F0000577269746520436FD6
:101960006E66696720423A0A000000005772697487
:101970006520436F6E66696720413A0A00000000E7
:101980002DE9FE4F0024DFF8709C0FF6741A0FF259
:10199000502B0FF2E40800F087F81D463CE000F001
:1019A000D1FA38E0002DFAD1404601F0D5F9397866
:1019B00000F0D0FB797800F0CDFB00F0CAFBF9789D
:1019C00000F0C8FB397900F0C5FB797900F0C2FB63
:1019D000217800F018F961782BA001F0BDF900BF63
:1019E0002DA001F0B9F9B97B00F0B4FBF97B00F050
:1019F000B1FB397C00F0AEFB797C00F0ABFBB97C2D
:101A000000F0A8FBF97C00F0A5FB217800F0FBF8C2
:101A1000617800F0B3F934469DF80100844229DA78
:101A2000661C3146DFF8EC0B01F096F99DF80000DA
:101A30000428F0D100F0E2F84C432044012D00F5D9
:101A40009E7400F1A80712D1404601F085F939785B
:101A500000F080FB797800F07DFB00F07AFBF978EC
:101A600000F078FB397900F075FB7979CBE7022D2E
:101A700098D1B4E7BDE8F78F5265616420436F6E7B
:101A800066696720413A0A005045434572726F7299
:101A90003A25640A000000005265616420436F6EBD
:101AA00066696720423A0A008DF8010001918DF8BD
:101AB000002070472DE9FE4F0024DFF83C5B0FF655
:101AC000400A0FF21C1B0FF27C08DFF8489BFFF75F
:101AD000EBFF31E00FF23C2001F03EF92BE0661CF9
:101AE000314600F04BF99DF800000F28F2D1404636
:101AF00001F032F900F082F84C43044404F19C07F1
:101B00005846397801F028F9797800F023FB00F085
:101B100020FBF97800F01EFB397900F01BFB797986
:101B200000F018FB04F59E745046217801F014F97A
:101B3000A17B00F0A5FA34469DF801008442CEDB7B
:101B4000BDE8F78F5265616420446576696365205E
:101B50005349443A0A0000002DE9FE4F144600257F
:101B60000FF2E8360FF2700B0FF274080FF27809DB
:101B7000DFF8A0AA8DF80000019126E0304601F0C0
:101B8000EBF821E06F1C394600F03DF80E2CF5D142
:101B9000484601F0E1F800F031F84D43411901F5F4
:101BA00090754046297801F0D7F8697800F0DBFDA0
:101BB000A97800F0D8FDE97800F0D5FD297900F08A
:101BC000D2FD697900F0C6FA3D469DF800008542D5
:101BD000D8DBBDE8F78F0000307825580A0A0000EE
:101BE000307825582C200000577269746520436FA7
:101BF0006D6D20446174613A0A00000001984FF451
:101C0000A67170473178504601F0A6B82DE9FE4F15
:101C10000FF2B0032FA40FF2C8090FF2D40A0FF28B
:101C2000E00BDFF8F0890193002600F0A6FD43E009
:101C300038A001F091F83EE000F093FD9DF800001F
:101C40000E28F5D1584601F087F802984FF4A67196
:101C50004E43861906F193075046F97801F07CF857
:101C6000397900F08BF87979204601F075F83978E8
:101C7000019801F071F879782DA001F06DF8B9782C
:101C80002FA001F069F8B97930A001F065F8F97971
:101C900032A001F061F8397A34A001F05DF806F560
:101CA0009E760FF25C60317801F056F8317B0FF6CA
:101CB000604001F051F82E469DF801008642BBDBE2
:101CC000BDE8F78F46434F4D303A307825582C20E9
:101CD0000000000049434F4D323A307825580A0041
:101CE00049434F4D313A307825582C2000000000F0
:101CF00049434F4D303A307825582C2000000000E1
:101D00005265616420436F6D6D20446174613A0ACD
:101D10000000000057726F6E672052656769737428
:101D2000657220547970652053656C6563740A0090
:101D300046434F4D313A307825582C2000000000A2
:101D400046434F4D323A307825580A0044415441B9
:101D5000303A307825582C2000000000444154418E
:101D6000313A307825582C2000000000444154417D
:101D7000323A307825580A0001980178484600F038
:101D8000EBBF00002DE9F84F2DED028B82B000F083
:101D9000C0F90FF6A8390FF698380FF6843400F022
:101DA000AFF99FEDB28B019120E000F067F900F0F0
:101DB000D4F900F0B4F9B86900F05CF900F0A5F9C5
:101DC00000F0DEFF01F010F800F0B3F9F86900F060
:101DD00051F900F09AF900F0D3FF01F005F800F096
:101DE000ADF900F0B0F900F0B4F9374600F09DF914
:101DF000DBDBF7E02DE9F04F14460026220085B02A
:101E000008BF0C2503D0012C14BF022C0625029616
:101E10008DF800000491A5F1010A0FF65C380FF26D
:101E2000E04905E0B5A000F097FF0298401C029041
:101E300002989DF8001088427BDA411C0FF60830AA
:101E400000F08AFF029A04994FF4A6704243881862
:101E50000390002700F59E70019014E000F072F8E6
:101E600010E0022CFAD153EC102B791C0FF6243021
:101E700000F072FF574505D1FFF77EFF0198C17A48
:101E800000F071FC7F1CAF42CCDA039800EB4700F6
:101E9000210008BFB0F844B008D0012C08BFB0F84A
:101EA0005CB003D0022C08BFB0F868B00FFA8BF01A
:101EB00000F0BEFF00F0D4F800F062FF00F094FFE5
:101EC00041EC100B20001ED1082F03D100F034F894
:101ED0000126D7E7681E87420AD153EC102B0FF674
:101EE000842000F039FFFFF747FF0198417AC7E7E8
:101EF000300053EC102B0CBF791C39460FF68420B0
:101F000000F02AFFBEE7012CABD1042F02D100F074
:101F100013F8B7E7574553EC102B08D10FF64420C0
:101F200000F01AFFFFF728FF0198817AA8E7F91D52
:101F3000E4E705B0BDE8F08F53EC102B0FF610204E
:101F400000F00ABF01A000F007BF000057726F6EDB
:101F5000672052656769737465722047726F757088
:101F60002053656C6563740A000000002DE9F84F8A
:101F70002DED028B82B000F0CCF80FF640290FF661
:101F80002C280FF61C2400F0BBF89FEDB38B0191B9
:101F900025E000F073F800F0E0F8FFF72FFE4F4364
:101FA0000744B7F9280000F043FF00F0AEF800F056
:101FB000E7FE00F019FF00F0BCF8B7F92A0000F0C6
:101FC00037FF00F0A2F800F0DBFE00F00DFF00F09C
:101FD000B5F800F0B8F8F97800F0BCF8374600F032
:101FE000A4F8D6DB02B0BDEC028BBDE8F18F2DE981
:101FF000FE4F00F08EF80FF6E4190FF634180FF6C6
:10200000CC1400F0E9F826E000F038F800F0A5F86C
:1020100000F085F8786B00F02DF8DFF8BC28DFF8C9
:10202000BC3800F017FF00F0ABFE00F0DDFE00F062
:1020300080F8B7F9380000F0FBFE00F011F800F06E
:102040009FFE00F0D1FE00F079F800F07CF83979BD
:1020500000F080F8374600F068F8D5DBBDE8F78F70
:10206000DFF87C28DFF87C3800F0F4BE8DEDB5A0F9
:10207000F7C6B03E8003801300F0DABE7E1C314606
:10208000284600F069BE00002DE9F84F2DED028BC7
:1020900082B000F03EF80FF670190FF65C180FF6DC
:1020A000481400F02DF89FED928B019121E0FFF78D
:1020B000E5FF00F052F800F032F8F86A00F0D0F8CE
:1020C00000F023F800F05CFE00F08EFE00F031F826
:1020D000386B00F0C5F800F018F800F051FE00F081
:1020E00083FE00F02BF800F02EF8F97900F032F8BA
:1020F000374600F01AF8DADB74E700000A0A00003D
:102100000FF604058DF80000704753EC182B00F013
:10211000A1BE00270FF2F87B0FF2E41A7047019876
:102120004FF4A6714F43074470479DF80000874263
:10213000704702460B46404600F00EBE02460B4674
:10214000484600F009BE07F59E775046397800F002
:1021500003BEB978584600F0FFBD204600F0FCBD34
:102160002DE9FE4FFFF7D5FF0FF6CC090FF6B808A3
:102170000FF6A40400F030F829E0FFF77FFFFFF727
:10218000ECFFFFF7CCFFF86B00F06AF8DFF84827A8
:10219000DFF8543700F05EFE00F0F2FD00F024FEA0
:1021A000FFF7C7FF386C00F05BF8DFF83427DFF883
:1021B0003C3700F04FFE00F0E3FD00F015FEFFF7A6
:1021C000BDFFFFF7C0FF397AFFF7C4FF3746FFF7BF
:1021D000ACFFD2DBBDE8F78F0FF22C758DF8000055
:1021E000019170472DE9F84F2DED028B82B0FFF77A
:1021F00090FF0FF660090FF630080FF64804FFF75E
:102200007FFF9FED3D8B019121E0FFF737FFFFF747
:10221000A4FFFFF784FF386A00F022F8FFF775FF8C
:1022200000F0AEFD00F0E0FDFFF783FF786A00F0FC
:1022300017F8FFF76AFF00F0A3FD00F0D5FDFFF7E8
:102240007DFFFFF780FFB979FFF784FF3746FFF77F
:102250006CFFDADBC6E600002D431CEBE2361A3FCA
:102260000002001200F0E4BD2DE9F84F2DED028BC5
:1022700082B000250FF2986B0FF2840A0FF6000966
:102280000FF2EC780FF2DC748DF800009FEDE28B1A
:10229000019127E0FFF761FFFFF7B0FC69434618A3
:1022A00006F1740706F59E7697F9000000F028FB0A
:1022B000FFF72BFF00F064FD00F096FDFFF739FFFC
:1022C00097F9010000F01CFBFFF71FFF00F058FD1D
:1022D00000F08AFDFFF732FFFFF794FC7179FFF7FA
:1022E00039FF6D1C9DF800008542D3DB7AE60000C3
:1022F0002D431CEBE236EA3E8DEDB5A0F7C6803EDD
:1023000043436F756E743A25642C00002DE9F84F35
:102310002DED088B84B00FF294770FF2F4580FF282
:10232000A4790FF2787B0FF2687A019700269FED6F
:10233000B38B9FEDB49B9FEDB5AB9FEDB9BB00F0A8
:102340001CFA1C46A5E0FFF7FDFDA1E0002CFAD128
:10235000504600F001FDB7F9000000F069FD00F003
:1023600077F900F00DFD00F03FFD00F066F9788888
:1023700000F042FE53EC1A2B00F06CFD00F054F913
:1023800000F035F953EC182B00F044FE00F050F942
:10239000B7F9040000F04CFD00F05AF900F0F0FC31
:1023A00000F022FD00F040F900F04CF90FF220702F
:1023B00000F0D2FC00F05AF900F053F900F04CF9AB
:1023C000797A0FF2487000F0C7FC0FF2507000F0FD
:1023D000C3FC00F0CBF900F0B7F900F0AEF900F063
:1023E000A5F900F09CF900F093F900F08AF900F0EB
:1023F00081F900F078F900F06FF900F0ACF9B97BE1
:102400000FF2C07000F0B5F900F05FF900F056F976
:1024100000F04DF900F044F900F03BF900F032F91A
:10242000B97B0FF6080000F099F9F97B0FF60C0064
:1024300000F09FF900F01FF900F0D3F800F08CFCD9
:102440000FF6240000F088FC397C0FF66C0000F0D9
:1024500083FC0FF6300000F07FFC797C0FF6300033
:1024600001F00F0100F078FCB97C0FF6300001F0AC
:102470003F0100F071FCF97C0FF62C0001F00F0118
:1024800000F06AFC3178FFF779FC717B00F06BF9A2
:102490002E469DF80100864280F29E80751C2946DA
:1024A0000FF2644000F058FC9DF800000C28EFD1BA
:1024B00002984FF4A6714E433044012C00F59E76ED
:1024C00000F176072ED1504600F046FCB7F9000027
:1024D00000F0AEFC00F0BCF800F052FC00F084FC10
:1024E00000F0ABF8788800F087FD53EC1A2B00F071
:1024F000B1FC00F099F800F07AF853EC182B00F0DA
:1025000089FD00F095F8B7F9040000F091FC00F0A7
:102510009FF800F035FC00F067FC00F085F800F053
:1025200091F8AFE7022C0DD10FF2A45000F014FC8B
:1025300000F09CF800F095F800F08EF8797A0FF230
:10254000CC509DE7032C39D10FF2D05000F004FCA1
:1025500000F00CF900F0F8F800F0EFF800F0E6F801
:1025600000F0DDF800F0D4F800F0CBF800F0C2F88D
:1025700000F0B9F800F0B0F800F0EDF8B97B0FF218
:10258000446000F0F6F800F0A0F800F097F800F0D2
:102590008EF800F085F800F07CF800F073F8B97B55
:1025A0000FF2886000F0DAF8F97B0FF2906000F02B
:1025B000E0F800F060F800F014F861E7042C07D1AF
:1025C0000FF2A46000F0C8FB397C0FF2A86057E757
:1025D000052C7FF4BBAE3CE704B0BDEC088BBDE836
:1025E000F18FF87BC0F380010FF26C607047C04A36
:1025F000C04B00F0CDBD0000102900080000000015
:10260000001071C0000000000000F83F613255303A
:102610002AA9233F082900087B14AE47E17A743FBA
:102620002D431CEBE2361A3F53EC192B00F0F2BCA1
:10263000024601980B4600F08FBB02460B465846F7
:1026400000F08ABB02460B460FF26C4000F084BBE0
:1026500053EC1B2B00F0FEBB397A0FF2A04000F0C8
:102660007BBBF9790FF2844000F076BBB9790FF2A9
:102670006C4000F071BBF87BC0F340010FF2C85012
:1026800000F06ABBB87BC0F380110FF2905000F0ED
:1026900063BBB87BC0F340110FF2705000F05CBB1D
:1026A000B87BC0F300110FF2585000F055BBB87B57
:1026B000C0F3C0010FF23C5000F04EBBB87BC0F33A
:1026C00080010FF2205000F047BBB87BC0F34001FF
:1026D0000FF2005000F040BB787BC0F380110FF286
:1026E000C44000F039BB787BC0F340110FF2A44026
:1026F00000F032BB787BC0F300110FF28C4000F089
:102700002BBB787BC0F3C0010FF26C4000F024BB00
:10271000B87AC0F301110FF2544000F01DBBB98923
:102720000FF23C40C1F30A0100F016BBB87AC0F3C7
:10273000C0010FF21C4000F00FBBB87AC0F380015B
:102740000FF2004000F008BBB87AC0F340010FF26E
:10275000E43000F001BB797B0FF25840C90900F06A
:10276000FBBA751C2946404600F0F6BAB97A0FF25A
:10277000B83001F0010100F0EFBA8DF801000291CC
:102780008DF80020704710B50FF23C505A4C00F005
:10279000E3FAFFF7E2FC04F1640000F0DDFA04F173
:1027A000C80000F0D9FA04F5967000F0D5FA04F5E7
:1027B000C87000F0D1FA04F5FA7000F0CDFA04F513
:1027C000167000F0C9FA04F52F7000F0C5FA04F590
:1027D000487000F0C1FA04F5617000F0BDFA04F52C
:1027E0007A7000F0B9FA04F24C4000F0B5FA04F542
:1027F000966000F0B1FA04F2145000F0ADFA04F55E
:10280000AF6000F0A9FA04F2DC5000F0A5FA04F57C
:10281000C86000F0A1FA04F2A46000F09DFA04F58B
:10282000E16000F099FA04F26C7000F095FA04F59A
:10283000FA6000F091FA04F6340000F08DFA04F624
:10284000980000F089FA04F6FC0000F085FA04F51F
:10285000166000F081FA1DA000F07EFA0FF28440AD
:1028600000F07AFA0FF2904000F076FABDE81040DE
:1028700017A000F071BA01460FF2944000F06CBA54
:1028800080B500F0D5FA00221C4B00F081FC00F06E
:1028900077FA00F0A9FA0B46BDE8024002460FF2B3
:1028A000784000F059BA411C0FF2884000F054BA49
:1028B00010B50446214607A000F08EFD21680FF2F6
:1028C0008840BDE8104000F047BA00000A00000050
:1028D0000A0A0000256400008DEDB5A0F7C6B03EE1
:1028E0002D431CEBE2361A3FF7C6803EE236EA3E45
:1028F000B81E85EB51B87E3FE0B300080040EF40C2
:102900004006401600F094BA494325643A0A000094
:102910005045434572726F723A25640A0A000000FE
:10292000526561642043757272656E743A0A0000E4
:1029300049313A25666D562C2000000049323A256F
:10294000666D560A00000000494325643A200A00DB
:10295000565245463241203D2025372E34665620BA
:102960000A000000565245463242203D2025372EAF
:10297000346656200A0000005045434572726F725B
:102980003A25640056253264203D2025372E3466D2
:1029900056200A00562564523D256656200A00003E
:1029A0005265616420564241543A0A0056424154ED
:1029B000313A202566562C20000000005642415432
:1029C000323A202566562C200000000052656164D2
:1029D0002049564241543A0A0000000056424154F0
:1029E000312566562C2000005265616420417667CF
:1029F000566261743A0A00005642314156473A2500
:102A000066562C20000000005642324156473A25B7
:102A100066562C20000000005265616420417667F4
:102A200049566261743A0A0049314156473A25666F
:102A30006D562C2000000000564231415647256655
:102A4000562C2000526561642041766743723A0A31
:102A50000000000049324156473A25666D562C2049
:102A60000000000052656164204F43523A0A0000A2
:102A70004F4331523A2025666D562C20000000004D
:102A80004F4332523A2025666D562C20000000003C
:102A900053746174757320413A0A000056524546DA
:102AA000315032353A2566562C20000049544D509D
:102AB0003A2566B0432C200056524547323A2566E7
:102AC000560A000043436F756E743A25642C20004B
:102AD00053746174757320423A0A00004F43314DBC
:102AE000494E3A307825582C200000004F43314D94
:102AF00041583A307825582C200000004F43324D81
:102B0000494E3A307825582C200000004F43324D72
:102B100041583A307825580A000000005374617417
:102B2000757320433A0A00004F4331413A3078250B
:102B3000582C20007E4F4331413A307825582C20C4
:102B4000000000004F4332413A307825582C2000D5
:102B50007E4F4332413A307825582C200000000047
:102B600043543A307825582C200000004354533AFF
:102B7000307825580A00000056415F4F563A3078A9
:102B800025582C200000000056415F55563A3078F9
:102B90002558200056445F4F563A307825582C204F
:102BA0000000000056445F55563A307825582C20D6
:102BB000000000004F5450315F45443A30782558AA
:102BC0002C2000004F5450315F4D45443A30782559
:102BD000582C20004F5450325F45443A30782558E5
:102BE0002C2000004F5450325F4D45443A30782538
:102BF000580A00005644453A307825582C200000E9
:102C0000564445313A307825582C2000494E5359C6
:102C10004E433A307825582C200000005350494646
:102C20004C543A307825582C20000000534C454530
:102C3000503A307825582C20000000005448534466
:102C40003A307825582C2000544D4F4443484B3A95
:102C5000307825582C2000004F534343484B3A30DE
:102C60007825580A0000000053746174757320447D
:102C70003A0A00004F435F434E54523A3078255889
:102C80002C20000053746174757320453A0A0000CB
:102C90004750494F3A307825582C200047504F3A3A
:102CA000307825582C2000005245565F49443A3070
:102CB0007825580A000000004F435F434E54523AB3
:102CC000307825580A0000004C697374206F662024
:102CD0004144424D533239353020436F6D6D616E42
:102CE000643A0A005072696E742027302720666F9C
:102CF00072206D656E750A00506C656173652065A4
:102D00006E74657220636F6D6D616E643A200A00A7
:102D100025730A0A0000000041646320436F6E7649
:102D2000657273696F6E2054696D65203D2025665C
:102D30006D730A00526573756C7420436F756E7401
:102D40003A25640A00000000456E74657220636DC8
:102D5000643A25640A0000000EB4C0B5024603A818
:102D600000210190009101AB0121044878440C300E
:102D700000F044FB06BC5DF810FB00BFD59A0000D4
:102D800001F000428B1AA3F16051B1F5801F0ADBFC
:102D9000B1F17F6F1FD242EAC102C10071F100415F
:102DA00042EB507070470B15C3F10903212B10D271
:102DB000890241EA905180020128494141F00041D5
:102DC00021FA03F0C3F12003994071F10041504111
:102DD0007047100070476FF0000013EB103F5CBFAE
:102DE000000E42EAC0507047C0F3C75181B1FF29BD
:102DF00006D0C110400721F0E04101F16051704759
:102E000041020CBF40F4E0016FF000410020704728
:102E100000F0004100020AD0B0FA80FC00FA0CF089
:102E200001F16051A1EB0C5101EBD021400570473D
:102E3000C11768B14840401AB0FA80F29040D21CE5
:102E4000C907C2F5846241EA025202EBD021400573
:102E500070474300B0B581EA030C0CF0004C40F21F
:102E6000FF7515EA11541DBF15EA1357AC42AF4266
:102E700039E0E41923EA455343F48013C90241F0D1
:102E8000004141EA505EC7021100A7FB0202002880
:102E90004FF00000EEFB01204FF00001E3FB0721A3
:102EA00018BF42F00102401800214941E3FB0E0126
:102EB000A4F580640F0302D252004041494154F10D
:102EC00001046CDD470872F1004250F1000051EB43
:102ED0000451A1F580115CBF41EA0C01B0BD4CEA80
:102EE00005510020B0BD05EA1357AC4214BFAF42F4
:102EF00041E050EA410E1CBF52EA430E02E0614637
:102F00000020B0BD24423C441BD15FEA070EF6D03E
:102F1000090302BF01460020AEF1140EB1FA81F799
:102F2000AEEB070401FA07FE0C37C7F1200100FAE7
:102F300007F7C8404EEA000E23EA455343F48013D6
:102F4000A2E733F00043B3FA83F704BFB2FA82FE7C
:102F500077440B3FE41BB7F1200E2FBF02FA0EF3AC
:102F6000BB40C7F1200E22FA0EFE38BF43EA0E0323
:102F7000BA40641C82E750EA410E14BF52EA430E85
:102F80006FF000014FF4001717EB430F8ABF19468B
:102F900017EB410FB5E74CEA05510020B0BDD4F165
:102FA0000104B4F120070FDAC4F12007520828BF4A
:102FB00042F0010210FA07F501FA07F7E1BF2A43D0
:102FC000E0403843E1400FE0352C98DCC7F12004A5
:102FD00052EA400220FA07F218BF42F0010231FA29
:102FE00007F0A1400A43002172F1004250F10000B5
:102FF00051EB0C01B0BD0000014648B1B0FA80F1C0
:103000008840C91CC1F58461090501EBD021400548
:103010007047000070B44FF0004591EA030F41F192
:1030200059826B40841A71EB030604D26E40001B78
:10303000B141121973414FF4001C1CEB410F34BF16
:103040007CEB430683E00C0DA4EB1356362E00F305
:103050007C80012E45EAC32341DC43EA525312BF70
:10306000D20292025B08240545EAC12141EA50518F
:10307000D2EBC020994125D407D1B0FA80F610FADE
:1030800006F162D00020203608E0B1FA81F6B140A6
:10309000C6F1200220FA02F21143B0404FEAF47464
:1030A000B4EB465434F001064FEA74040AD8D6F55E
:1030B0000016760D04F00044F04061FA06F250402C
:1030C000F1404840C00A40EA415021F0004128BF89
:1030D0005FEA500550F1000044EBD12135E0DB0AF6
:1030E00045EAC121C90AB6F120050EDD42EA0242D5
:1030F000120CC5F1200603FA06F6EB4042EA06057B
:103100006D42984161F100010DE062FA06F5F2406E
:10311000554063FA06FC82EA0C02F3405A406D42C5
:10312000904161EB030111F4801F05D1641E62051B
:1031300002D06D004041494121F48011430875F1EE
:10314000004350F1000041EB045170BC70471CEB90
:10315000410F15D223F0004352EA43060BD04FEA49
:103160004C0CBCEB410F04D80C0D661E342EB7DDA1
:10317000EBE7801A994150EA410608BF0021E4E7D5
:1031800008BF1CEB430F28BF6FF00001DDE7000014
:10319000F0B540F2FF7581EA030C0CF0004C15EA23
:1031A00011541DBF15EA1357AC42AF42E5E0BC41D4
:1031B000C1F31301C3F31303801A994143F480133D
:1031C00004D2641E4000494180185941C90241EAB5
:1031D0005051B1FBF3F603FB1611A2FB0675D7EBBA
:1031E000C020A94102D2761E80185941C90241EA85
:1031F0005051B1FBF3FE03FB1E11A2FB0E75D7EB82
:10320000C020A94103D2AEF1010E801859418902B4
:1032100041EA9051760546EA8E2EB1FBF3F603FBA8
:103220001611A2FB0675D7EB8020A94102D2761EAB
:1032300080185941C90241EA50514EEA060EB1FBCD
:10324000F3F603FB1611A2FB0675D7EBC020A941CC
:1032500002D2761E80185941C90241EA5051B1FB91
:10326000F3F703FB1711A2FB0735D3EBC020A941ED
:1032700067F100070CBF004247F0010766F3D5274E
:103280004FEA1E31B80814F5806412DDBD0775F1F0
:10329000004250EB0E5051EB045111F5801F5CBF02
:1032A00041EA0C01F0BD4CF07F6141F0E0410020AB
:1032B000F0BDBD076D0840EA0E5041F48011D4F115
:1032C0000104B4F120060ADAC4F120060200E0404D
:1032D00001FA06F3E1401843B24015430EE0342CE6
:1032E00013DCC6F1200445EA40056D0820FA06F219
:1032F000154321FA06F0A1400D43002175F100426B
:1033000050F1000051EB0C01F0BD00205FEA0C0110
:10331000F0BDCFB992185B41B3FA83F704BFB2FA9C
:1033200082F6BF190B3FB7F120062FBF02FA06F352
:10333000BB40C7F1200622FA06F638BF3343BA4035
:103340001CB1E419641E33E77F4231F00041B1FA49
:1033500081F404BFB0FA80F6A4190B3CB4F1200646
:103360002FBF00FA06F1A140C4F1200620FA06F6AC
:1033700038BF3143A0403C1B1AE7AC421ABF05EAF4
:103380001357AF4212E050EA41061CBF52EA43060F
:10339000BFE750EA4107304661461CBF41EA05518C
:1033A000F0BD52EA430C08BFC143F0BD00204FF40A
:1033B000001616EB410F98BF16EB430F08BF16EB34
:1033C000410F24BFC14305E016EB430F0CBF61461C
:1033D0004CEA0551F0BD00000EB4C0B5024603A88A
:1033E00001900021009101AB034878440A3001F0BC
:1033F00003F906BC5DF810FB9D9400002DE9F14F28
:10340000B2B09946924600230691CDE900333C9A2A
:103410000F930DF14A0114914A7011E0329E574604
:103420002C4617F8011B0698B0470028069000F0BC
:1034300026810F98401C641E0F90F2D13296AA4448
:103440009AF80000252808D10021002209910A924B
:103450000B910C920D910E920FE06A464FF0FF31E6
:10346000504602F0AAF8050002D10F9800F066BE9F
:10347000D4D50125E3E741F001011AF8010F202816
:10348000F9D023280CD02B2804D02D2805D03028A3
:1034900009D00BE041F00201EFE741F00401ECE755
:1034A00041F00801E9E741F01001E6E72A280FD1D1
:1034B000D9F8002052F8040BC9F800200028119018
:1034C00003D54042119041F004010AF1010A14E0D1
:1034D0001192DFF8EC3B0AE01198984205DA00EB14
:1034E000800402EB4402303A11920AF1010A9AF880
:1034F0000020A2F130000A28EED39AF800002E280E
:1035000003D04FF0FF32109229E01AF8010F2A2859
:1035100009D1D9F8000050F8042BC9F80000109226
:103520000AF1010A1BE02D280CBF0AF1010A002054
:1035300000221092DFF8882B0BE040B9109B9342D9
:1035400005DA03EB830504EB4504303C10940AF1E3
:10355000010A9AF80040A4F130030A2BEDD3ADF82C
:1035600048100FF660309AF8001002F037F808B1F2
:103570001AF8010B8DF84A009DF84A00682805D119
:103580009AF8000068280CD1622106E06C2804BF7C
:103590009AF800006C2804D171218DF84A100AF1C4
:1035A000010A1FA808901AF801BBBBF125012DD014
:1035B0001C3900F06181091F022940F25D810E393A
:1035C0002AD0491F00F0B284093900F05581891EC4
:1035D00000F04885491E00F0F484491E022940F29B
:1035E0004B81091F00F0ED84491F00F0BA80491E8D
:1035F00000F09C84491E65D0C91E21D0891E00F0B0
:103600009584C91E00F0928400F04BBD25238DF8EF
:103610007C30012109912AE06C208DF84A00D9F80C
:10362000000050F8042BC9F80000002A43D1149977
:10363000487800283DD04FF0FF340FF6902012E07C
:103640009DF84A006C28EAD0D9F8000050F8044BE5
:10365000C9F800000794D4B91499487898B14FF08C
:10366000FF340FF6842001F0C5FF201A07D13298ED
:103670001FAA04A900F065FD00287FF5E1AE4FF018
:10368000FF3000F05BBD0FF67C200790EFE7109D48
:10369000002D04D5204601F0CDFF044607E02A4660
:1036A000204601F0E3FF002814BF041B2C460A94B7
:1036B000DDE70FF65422329804A900F0C8FD002877
:1036C000D5D5DCE7D9F8001051F8040BC9F8001083
:1036D00020F00004002121F0FF351FABCDE90445A7
:1036E0000793DDE9042308993C2413B90AB910981B
:1036F00098B102F00F053035641EEEB23A2EA8BF25
:103700002735120942EA03721B090D5508BF002A2A
:1037100003D007980D19A842EBD308190790C4F1FC
:103720003C0210980A92824209DABDF84810821AC7
:103730004FF6EF7001400C92ADF8481097E7002863
:1037400095D59DF8480000F0140010288FD1119BEA
:1037500009990C985B1A1B1A9A1A002A87DD0C9299
:1037600085E71499487820B14FF0FF340FF69C108C
:1037700079E79DF84A00622862D0682819D06A2843
:1037800040D06C2806D071284DD074282DD07A28CE
:103790001ED064E0D9F8001051F8040BC9F80010ED
:1037A00020B94FF0FF340FF67C105CE70F990160F1
:1037B0005DE7D9F8001051F8040BC9F8001020B9E2
:1037C0004FF0FF340FF65C104DE70F9901804EE784
:1037D000D9F8001051F8040BC9F800100028E5D101
:1037E0004FF0FF340FF63C103DE7D9F8001051F8C8
:1037F000040BC9F800100028D8D14FF0FF340FF6A1
:10380000241030E7D9F8001051F8040BC9F8001063
:1038100020B94FF0FF340FF60C1024E70F9AD3179E
:10382000C0E9002323E7D9F8001051F8040BC9F8C8
:1038300000100028F2D14FF0FF340FF6E80012E735
:10384000D9F8001051F8040BC9F8001020B94FF056
:10385000FF340FF6D00006E70F99017007E7D9F89B
:10386000001051F8040BC9F8001000289ED14FF049
:10387000FF340FF6B000F6E6D9F80020D21D22F092
:103880000702C9F80020D2E900010832C9F8002077
:10389000CDE90401C80F02D009982D210AE0BDF836
:1038A0004800810702D509982B2103E0C00705D500
:1038B000099820211FAA1154401C09901FA809999A
:1038C0004BF020024318DDE90401CDE92E01612A05
:1038D000079315AC0BD01098002802D50620109045
:1038E00005E001BF4BF02000672801211091DDE9C0
:1038F000040148004015401C0A4611D109030FD0AD
:10390000ABF1610503201A2D0A9002D20FF6A03107
:1039100001E00FF6A0310322184601F0D3FEA6E61F
:1039200050B9120308D1ABF1610503201A2D0A909A
:1039300016D30FF68831EEE7DDE90401CDE9300159
:10394000DDE9302323F00047B7F5801F22F00006A1
:103950000DD20022002F08BF002E029203D116E0E4
:103960000FF65431D7E702AA01F0B8FE0FE0DFF8F6
:10397000F00ADFF8F01A00EB17500290DDE930236F
:103980004FF0FF301940DFF8E07A10403943CDE9BD
:1039900004014BF0200061280DD1079830210170FF
:1039A000821CBBF1610F07920CBF78215821417036
:1039B0000998801C0990DDE9040120F0000231F033
:1039C000004308BF002A02D10026002571E14BF018
:1039D0002008B8F1610F40F0BE801098002847BF62
:1039E00021210391401C0390039FDDE92E017F1CE0
:1039F00000220023DDE9044501F0A8FE02998DF8BC
:103A0000542038BF85F00045091F002F02910DF1A9
:103A100055065DDDDFF8541ACDE9302140F2FF7321
:103A20002E93204629460022002301F0A7FE4FD204
:103A30004800400D00F11C0315D0002B13DD2E981B
:103A400083420ADBDDE9300121F0004005F000424D
:103A50000243DDE93001114611E06FF31E5141EAE6
:103A6000035120460BE024F0000035F0004108BF70
:103A700000280FBF29461C22294601F097FE044664
:103A80000D4601F031FFFF1F002F804609DDFFF7D3
:103A9000CFF902460B462046294600F013FD0446A6
:103AA0000D46F01D0721B8F1000F0CDD491E5EBF69
:103AB00008F00F0200F8012D4FEA2818F3D502E0B4
:103AC000002200F8012D491EFAD5C61D002FA8DCE2
:103AD0000DF15500361A03988642D8BF30460028AB
:103AE0000DF1550430D4B04206DA0DF155010A5CEF
:103AF000082AA8BF0F2100DA0021024615AB1344A3
:103B000000E0401E13F80159521E8D42F9D00F29D2
:103B100004D10DF155018B5C5B1C8B54002A04D53C
:103B20000299091D15AC401C0291411E0CD462186B
:103B3000ABF13A0613783033DDB23A2DA8BFF31853
:103B4000491E02F80139F5D51099002940F1AF80DE
:103B5000421E1092ABE00299DFF8142947F2975009
:103B6000414391FBF2F2DDE92E45029225F000453A
:103B7000D2F1070204DD2046294600F04DFC0BE09F
:103B800052420020DFF8EC1800F046FC02460B46DB
:103B900020462946FFF7FCFA0446B8F1660F109854
:103BA00006BF029F0A3706273F18142FC8BF1427E5
:103BB00030208DF854000D460020DFF8BC18CDE908
:103BC0002E010DF15506002F33DD2046294601F068
:103BD000A9FE01460A4606F1080304200A26B2FBA4
:103BE000F6F606EB860EA2EB4E02303203F8012CFD
:103BF0000A22B6FBF2F202EB820EA6EB4E0630363C
:103C0000401E03F8026DE9D1083F002F03F10806BA
:103C1000D9DD0846FFF7F0F902460B462046294653
:103C200000F050FCDDE92E23FFF714F904460D46A1
:103C3000CBE70DF15500361A0DF1550404E002985A
:103C4000401E761E0290641C20783028F7D0B8F110
:103C5000660F02D10299491C04E0B8F1650F0CBF50
:103C600001210021109808188642B8BF701E002854
:103C70001DD4B04204DA215C3429C8BF392100DCEC
:103C800030210246631E9D1800E0401E15F80169B0
:103C9000521E8E42F9D0392902D1A15C491CA1548F
:103CA000002A04D50299491C1C46401C0291064674
:103CB000029D01F08CFC406A0778DDF8408030B24C
:103CC000002802DC01260FF2F8744BF02000662871
:103CD00008BF6D1C16D0672846D128B210F1040F1A
:103CE00048DB404546DA9DF848006D1C010703D4C7
:103CF00030B24045B8BF804628B2B8EB000848BF94
:103D00004FF000080FFA85FB07980A99BBF1000FE6
:103D100000F3B2804A1C0A9230234354B8F1000FDA
:103D200003DC9DF84800010704D50A98411C0A915C
:103D300007990F5418EB0B0FB8BFC8F100052DB24F
:103D400068420D90A84432B29045B8BF4646079BE2
:103D50000A9836B20B9632462146184401F0B2FC5E
:103D6000A8EB06000E90CBE0BBF1610F17D14FF02E
:103D7000700B19E030B2404504DA9DF848100A078C
:103D800058BF8046B8F1010848BF4FF00008BBF1AA
:103D9000670F14BF4FF0450B4FF0650B04E0BBF10C
:103DA000410F08BF4FF0500B0A98411C0A91B8F11F
:103DB000000F079914F8012B0A5403DC9DF8480002
:103DC00001071AD50A98411C0A91B8F1000F07990A
:103DD0000F5412DD761E30B2804507980A9BB8BF9B
:103DE000464632B22146184401F06CFC0A9936B2BC
:103DF00071180A91A8EB06000D9007980A990844DB
:103E00002AB2002A80F800B003D42B224270811C11
:103E100004E02D2141701546811C6D4200202EAA20
:103E20000A2409E02B4693FBF4F505EB8506A3EB8A
:103E3000460302F8013B401C2DB2002DF2DC0128A4
:103E400006DC4BF02002652A04BF302201F8012B6A
:103E500000282EAA08D1302001F8010B06E0401EF0
:103E6000135C303301F8013B0028F8DC079A0A980C
:103E70001044091A0B9143E0084431B22AB291422E
:103E800019DA32B2214601F01DFC0A9936B27118D6
:103E9000ABEB0606B8F1000F0A910D9603DC9DF816
:103EA0004800020704D5079847540B99491C0B9109
:103EB000CDF8388024E0214601F004FC0A98761BF6
:103EC0005844B8F1000F0A9003DC9DF848100A0727
:103ED00003D5411C0A9107990F5430B280450798C9
:103EE0000A9BB8BF464632B204EB0B01184401F0FE
:103EF000E9FB0A9836B230180A90A8EB06000D903C
:103F00009DF8480000F0140010287FF4B0AB099A27
:103F10000A990D988A180B9982180E988A18821897
:103F200011988242BFF6A3AB821A18E49DF84A00AA
:103F3000622808D068280ED06A2814D06C281FD0B8
:103F4000712810D01CE0D9F8001051F8040BC9F802
:103F50000010C0B21AE0D9F8001051F8040BC9F8EB
:103F6000001080B212E0D9F80020D21D22F0070222
:103F7000C9F80020D2E900010832C9F8002006E0A3
:103F8000D9F8001051F8040BC9F800100021CDE950
:103F900004019DF8480001075AD5DDE90423002BF0
:103FA00008BF002A54D04BF02000782850D109983F
:103FB0001FA930220A54401C431C099301F800B089
:103FC00046E09DF84A00622808D068280ED06A288A
:103FD00014D06C281FD0712810D01CE0D9F8001024
:103FE00051F8040BC9F8001040B21AE0D9F80010DB
:103FF00051F8040BC9F8001000B212E0D9F8002003
:10400000D21D22F00702C9F80020D2E900010832CF
:10401000C9F8002006E0D9F8001051F8040BC9F8DF
:104020000010C117CDE90401002902D509982D21FE
:104030000AE0BDF84800810702D509982B2103E06A
:10404000C00705D5099820211FAA1154401C0990CA
:104050001FA809990144079104A8594600F057F98F
:10406000FFF705BB9DF84A006C280BD00121099190
:10407000D9F8000050F8041BC9F800008DF87C1036
:10408000FFF7F5BAD9F8000050F8041BC9F8000092
:1040900015914FF0FF3210920021169115AAFFF7EB
:1040A0000ABB25210122BBF1000F8DF87C1009927B
:1040B0003FF4DDAA8DF87DB00221FFF7ABBA000016
:1040C000CBCCCC0C686A6C747A4C00007072696E50
:1040D00074665F733A2062616420256C732061729C
:1040E00067756D656E7400007072696E74665F73DB
:1040F0003A2062616420257320617267756D656E78
:104100007400000000000000000000007072696E82
:1041100074665F733A20256E20646973616C6C6FFE
:10412000776564007072696E74663A20626164201B
:10413000256E20617267756D656E740033B0BDE8E1
:10414000F08F2DE9FC410F46064690467A6B786960
:10415000396ABC6A121AB869521A796A121AF8696D
:10416000521A121A97F83800141B41070FD4202056
:10417000002C8DF800000ADD254601236A463946E9
:10418000304600F07DF900285DD16D1EF5D17B69C8
:1041900042463946304600F073F9002853D13020AA
:1041A0008DF800003D6A002D09DD01236A4639467D
:1041B000304600F065F9002845D16D1EF5D1BB6988
:1041C000FA683946304600F05BF900283BD13020D0
:1041D0008DF800007D6A002D08DD01236A4639460E
:1041E000304600F04DF970BB6D1EF6D1F868B96924
:1041F000FB6942183946304600F042F918BB3020BE
:104200008DF80000BD6A002D08DD01236A4639469D
:10421000304600F035F9B0B96D1EF6D197F8380088
:1042200041070DD52020002C8DF8000008DD01236A
:104230006A463946304600F023F920B9641EF6D1AB
:104240000020BDE8F6814FF0FF30BDE8F6812DE992
:10425000F8470D46A3B02F6B002F8246904648BF0B
:104260006FF0004701F072FB696B401801AA002152
:10427000C2E90011812828BF4FF0FF3044D289469F
:104280001EE0A74230DB6869201881280BD300218B
:10429000696303AA29465046FFF753FF5FEA000906
:1042A00022D40020686103AB6E69224669469819E2
:1042B00001F008FAA6196E6158F8040BA0B13F1B73
:1042C000002F11DDD8F8001001AA684601F07DF931
:1042D0000446002C05D4D8F800000028D1D1641E73
:1042E000CFD54FF0FF390EE0B9F1000F504604D1A1
:1042F00003AA2946FFF725FF8146B9F1000F02D135
:10430000002068616863484624B0BDE8F0872DE965
:10431000FC4307466F293E6908BF082405D041F0D9
:104320002000782814BF0A2410243C25D7E9002354
:10433000642918BF69299046994605D1002B03D5F9
:10434000D8F1000869EB4909B9F1000F08BFB8F1CD
:10435000000F0CD1386B50B9082C39D197F83800C0
:10436000010735D530203B2586F83B0030E08DF83D
:104370000010404649462246E31701F0EDFA30327C
:10438000D0B26D1E3A28019504DB9DF80000A0F123
:1043900051018A187255404649462246E31701F0FA
:1043A000DBFA80465FEA010908BFB8F1000F03D0CD
:1043B000F86871198842DCD3082C09D197F83800C5
:1043C000010705D5705D302802D06D1E3020705574
:1043D000C5F13C02BA617119F960386B824208DAA2
:1043E000821A3A624FF6EF70398F01403987BDE883
:1043F000F38300280ED597F8380000F01400102839
:1044000008D17B6B7969386A5B1A1B1A9A1A002AE1
:10441000C8BF3A62BDE8F3832DE9D04306460F4694
:1044200014464FF00008DFF8549012E0E00707D57B
:1044300042464B4630463946FEF70CFD06460F46CF
:104440004046494642464B46FEF704FD641080460E
:104450008946002CEAD130463946BDE8D0830000B9
:1044600002FCFFFFFFFF0F800000E03F0000F07F35
:10447000A08601000000F03F84D79741000024404F
:10448000F8B505460E4617461C4600205CB117F8E5
:10449000011BB068A847B06030B1F06A401CF06200
:1044A0000020641EF3D1F2BD4FF0FF30F2BD0000DA
:1044B0006E616E004E414E00696E6600494E4600C8
:1044C0003000000070B44FF0004591EA030F7EF514
:1044D000A9AD6B40841A71EB030603D2001BB141F6
:1044E000121973414FF4001C1CEB410F34BF7CEBDD
:1044F000430442E00C0DA4EB1356352E4FDC45EA85
:10450000C323DB0A45EAC121C912B6F120050DDD3E
:1045100063FA05F6EB4086EA0305124218BF45F040
:104520000105C01851F100010CD213E062FA06F542
:10453000F2405540F3415A40B340F3405A4080188E
:10454000594107D349085FEA30005FEA350528BFC3
:1045500045F0010501F58011420875F1004250F166
:10456000000041EB04514E0016F5001F70BC38BF2F
:1045700070470020090D090570471CEB410F10D250
:1045800052EA43060BD0BCEB410F05D80C0DAB43F0
:10459000661E342EB6DD02E0AB438018594170BC74
:1045A000704770BC70470000034608460122C1688E
:1045B000491CC16000210068184703460846C168CD
:1045C0000269491C521E002A0261C16003D40068BE
:1045D0000122002118474FF0FF307047034608467C
:1045E0001146C268521E11F1010FC26002D000686C
:1045F00000221847704700002DE9F84F9CB008AE24
:104600000027C6E9007700914FF0FF341B68019343
:1046100002920DF14702269B8DF81F30A0460397AA
:104620001B92814602E10A98029D25280CBF771E45
:1046300037467F1E15D40398401C03900122009832
:104640000021C84715F8011B8842F2D0024669468E
:104650004846FFF7C3FF0020404580F28B8500F0FD
:1046600088BD02980A9930442529029008D1007823
:104670002A280ED10298401C029010F8011D09E072
:104680000A98002840F0D280404580F2738500F0FF
:1046900070BD00218DF81C1000210591DFF8DC3A77
:1046A0000AE00598984205DA00EB800601EB460126
:1046B00030390591501C0290029A1178A1F1300016
:1046C0000A28EED306940FF6B820117800F086FF82
:1046D00020B10298401C0290401E00788DF81D0009
:1046E0009DF81D00682805D10299087868280CD12A
:1046F000622206E06C2802BF029908786C2804D177
:104700007122491C8DF81D200291029801780FF644
:10471000782000F063FF80B90398401C03900122C9
:1047200000980021C847064601F099F90028F3D106
:10473000324669464846FFF751FF00208DF81E00BB
:1047400002980178253930D01C3900F0C980091F42
:10475000022940F2C5800E393BD0491F00F06B831F
:10476000C91E1FD0891F00F0BB80891E00F0ED8498
:10477000491E00F06083491E022940F2B180091FE2
:1047800000F05983491F2AD0491E012940F2538362
:10479000091F21D0891E00F04E83C91E00F04B83F3
:1047A00000F0E2BC224600F0D1BC0398401C03900C
:1047B00001220098C8470646252E2AD0324669466F
:1047C0004846FFF70BFF16F1010F40F0CD8400F0D3
:1047D0001DBC6C208DF81D00012200F0B7BC9DF8B7
:1047E0001C00B0B99DF81D0062286DD0682851D01A
:1047F0006A285BD06C2801D0712857D0019951F8F4
:10480000040B019118B90FF6881000F09ABC0399B7
:104810000160B8F1000F9DF81E0048BF4FF000087E
:1048200008B108F1010802994A1C029200210A917C
:1048300008AB029922460AA800F0C1FE0646002EE7
:1048400005DC029801784E1EB641F643F60F0A9831
:1048500001F00FF901F003F900283FF4E4AE0398EA
:10486000401C0390012200980021C847074601F030
:10487000F6F80028F3D13A4669464846FFF7AEFEFF
:1048800017F1010F7FF4EDAE5FEA080040F172848A
:1048900000F068BC019951F8040B019118B90FF6AA
:1048A000F00000F04EBC03990180B2E7019951F885
:1048B000040B019118B90FF6D80000F042BC039A1E
:1048C000D317C0E90023A4E7019951F8040B019123
:1048D00018B90FF6BC0000F034BC0399017098E7DA
:1048E00005980028D8BF6FF00040049069464846FC
:1048F000FFF763FE00262B2818BF2D280DF1300A84
:1049000007D18DF8300069464846FFF756FE0DF195
:10491000310A0A270025302818D169464846FFF792
:104920004CFE40F02001C9B2782902D00125294669
:104930000BE130208AF800008AF8011048466946E9
:10494000FFF73BFE0AF1020A1027F0E740F02001D2
:10495000CAB26E2A4CD16E200AF8010B694648464D
:10496000FFF72BFE83464BF020000027C0B26128E2
:1049700040F09A8161210AF8011B48466946FFF719
:104980001CFE83464BF02000C0B26E2840F08C81A4
:1049900069464846FFF711FE282806D002466946B8
:1049A0004846FFF71BFE6E2066E00498401E049008
:1049B00005D469464846FFF7F7FD834603E00399AF
:1049C000491C0391A346CDF828B0584601F06BF876
:1049D0000028EAD1ABF130000A28E6D30A985F2814
:1049E000E3D08346BBF1290F40F05E816E2043E0A7
:1049F000C9B2692940F0B08069200AF8010B694604
:104A00004846FFF7DAFD83464BF020000027C0B28E
:104A10006E2840F049816E210AF8011B0398049921
:104A2000401C491E00290491039005D400980122DE
:104A30000021C847834600E0A3464BF02000C0B2E7
:104A4000662840F0318103980499401C491E0029D2
:104A50000491039004D4009801220021C84700E08B
:104A6000204640F02001C9B2692908D002466946B3
:104A70004846FFF7B3FD66200AF8010B1AE10398D8
:104A80000499401C491E00290491039005D4009804
:104A900001220021C847834600E0A3464BF02000D6
:104AA000C0B26E2840F0008103980499401C491E52
:104AB00000290491039005D4009801220021C847E1
:104AC000834600E0A3464BF02000C0B2692840F0C6
:104AD000EB8003980499401C491E0029049103901F
:104AE00005D4009801220021C847834600E0A34670
:104AF0004BF02000C0B2742840F0D680039804998F
:104B0000401C491E00290491039005D400980122FD
:104B10000021C847834600E0A3464BF02000C0B206
:104B2000792840F0C18066210AF8011BC2E0039891
:104B3000401C0390204607E00498401E0490F6D4E1
:104B400069464846FFF730FD01213028F4D00D4674
:104B500011B130210AF8011B8346284600250EE0DA
:104B60000398401C0390A34608E00498401E04905C
:104B7000F6D469464846FFF717FD834601201BF12E
:104B8000010F1BD05FFA8BF2612AA8BFABF157016E
:104B90000ADA412AA8BFABF1370105DA303A0A2A0E
:104BA00034BFABF13001FF21C9B2B94206D2242D86
:104BB000BABF0AF801BB6D1C761CD6E78DF8280039
:104BC0000B9500F004FD406A01788B4510D10AF87E
:104BD00001BB03980499401C491E002904910390CD
:104BE00005D4009801220021C847834600E0A3466F
:104BF0000B98E8B99DF828000FE00398401C03903B
:104C0000A34609E00498761E401E0490F5D4694638
:104C10004846FFF7C9FC83460120BBF1300FF1D0B5
:104C2000002E8DF8280003D530200AF8010B761CE1
:104C30009DF828000B9D13E00398401C0390A346A9
:104C40000DE0242DBCBF0AF801BB6D1C0498401E6A
:104C50000490F1D469464846FFF7A6FC834601203C
:104C60001BF1010F14D05FFA8BF2612AA8BFABF1E0
:104C700057010ADA412AA8BFABF1370105DA303A09
:104C80000A2A34BFABF13001FF21C9B2B942D8D3EF
:104C9000054648B14BF020000A2FC0B235D1652837
:104CA00035D001E083460D465A4669464846FFF72F
:104CB00095FC15B300218AF800109DF81C0000280F
:104CC0007FF4A7AD0A2F0B4674DC32460CA801F026
:104CD00083F801228DF81E20019A9DF81D60131D96
:104CE0006C2E40F0938012680193002A40F08B8074
:104CF0006248784400F5C37023E20CA8824508BFDF
:104D00001BF1010F40F0308280E17028CCD10AF80D
:104D100001BB0498401E049010D40398401C0390DB
:104D2000012200980021C8472B2818BF2D2811D137
:104D30000AF8010B0498401E049004D50398401C07
:104D40000390204606E00398401C0390012200983F
:104D50000021C84700210DE00398401C0390204625
:104D600007E00498401E0490F6D469464846FFF7D1
:104D70001BFC01213028F4D00A001CBF30220AF8A5
:104D8000012B0025A0F130020A2A8BD2082DBCBFCE
:104D90000AF8010B6D1C0498401E049004D503987A
:104DA000401C0390204603E069464846FFF7FCFBA1
:104DB0000121E7E700220CA801F00EF8B2000E4630
:104DC00037467B005B0D02EB030511D0002D0FDD94
:104DD00040F2FF72954206DBDFF8B01606F000469F
:104DE0003143002075E76FF31E5747EA055170E71E
:104DF00020F0000631F0004708BF002E3FF469AFF5
:104E000000F0D4FC65E7C2E9000102E54C2E07D1B1
:104E100012680193002AF6D1184878445E3090E178
:104E2000166801931EB915487844503089E1FDF7A2
:104E3000A7FF3060EDE405980028CCBF401EDFF8E6
:104E4000500600280AAF049012D40398401C039027
:104E5000012200980021C8472B2818BF2D2816D101
:104E60008DF828000DF129070498401E049007D5FD
:104E70000398401C0390204609E000BF28780000FA
:104E80000398401C0390012200980021C847029A11
:104E900012780021642A18BF752A0FD0692A08BF2A
:104EA00000260CD06F2A08BF082608D0702A1CBF25
:104EB00042F02002782A02D1102600E00A2630288B
:104EC0002ED104980125401E0490039805D4401C5F
:104ED000039001220098C84702E0401C039020463E
:104EE00040F02001C9B2782917D1002E18BF102E2A
:104EF00027D104981026401E0490039807D4401C24
:104F00000390012200980021C847002519E0401CA9
:104F1000039025464FF0000A4BE096B9082610E0B2
:104F2000FEB90A261DE00398401C0390204607E0C6
:104F30000498401E0490F6D469464846FFF734FBB7
:104F400001253028F4D029460A000AD0302207F87B
:104F5000012B06E0401C0390012200980021C84765
:104F6000012110F1010F22D0C2B2612AA8BFA0F125
:104F700057030ADA412AA8BFA0F1370305DA303A0D
:104F80000A2A34BFA0F13003FF23DBB2F2B293420E
:104F90000DD21B998F4238BF07F8010B0498401EB1
:104FA00004900398D6D5401C039001212046054665
:104FB0008A462A4669464846FFF710FBBAF1000FB9
:104FC0001DD0002139709DF81C0000287FF421AC11
:104FD00002980078642818BF69286BD032460AA866
:104FE00001F0BEF801228DF81E20029A1378702B72
:104FF00011D1019B53F8042B01934AB99FE00AA8F1
:10500000874208BF15F1010F40F0AE802046ACE0AA
:105010001060FFF7FEBB9DF81D20622A3AD0682A77
:1050200011D06A2A26D06C2A06D0712A2AD0742A76
:1050300019D07A2A10D036E0019B53F8042B019343
:10504000002AE5D17BE0019B53F8042B0193002A51
:1050500075D01080FFF7DDBB019B53F8042B019343
:10506000002AD5D16BE0019B53F8042B0193002A51
:10507000CED164E0019B53F8042B0193002A7FF406
:10508000C2AE5CE0019B53F8042B0193002A7FF42D
:10509000BAAE54E0019B53F8042B0193002A4ED082
:1050A0001070FFF7B6BB019B53F8042B0193002A45
:1050B000AED144E032460AA801F0A6F801228DF8EC
:1050C0001E209DF81D20622AE4D0682ABBD06A2ADF
:1050D0001ED06C2A06D0712A22D0742A10D07A2AC7
:1050E00007D025E0019B53F8042B0193002A8FD1B0
:1050F00025E0019B53F8042B0193002A88D11EE080
:10510000019B53F8042B0193002A7FF481AF16E032
:10511000019B53F8042B0193002A7FF474AE0EE038
:10512000019B53F8042B0193002A7FF46CAE06E038
:10513000019B53F8042B0193002A7FF469AF0FF20F
:10514000743000F057FA201A04E0002269464846FD
:1051500000F04EF800283FF75CAB269929B110F11A
:10516000230F02D1204605E00020B8F1000F48BF10
:10517000804640461DB0BDE8F08F0000CBCCCC0C83
:10518000686A6C747A4C000063436E5B0000000038
:105190007363616E665F733A2062616420256E20DE
:1051A000617267756D656E7400000000C9B208E039
:1051B00003789942A4BF90F802C08C4513DAC01C52
:1051C000D21E032A0AD343782D2BF1D010F801CB3D
:1051D0008C4518BF521EF4D105E0521E2AB110F8BA
:1051E000013B8B42F9D1012070470020704700003D
:1051F0002DE9F04F8BB00D46002603968146697F5E
:10520000019204A86C2901990CBF4FF0010BB34621
:10521000C0E90066002924D5A868411CA960084699
:1052200001785E2903BF401CA86010F8014D0024DE
:10523000AF6838785D280CBF781C38465D2100F0D7
:10524000CDF9002800F01381C11B0091A8600098DF
:10525000022806DD821E2D21781C00F007FA00B11D
:1052600001266869002805DC0198002814BF6FF04A
:10527000004001202861287FD0B96868011D0068BE
:105280006960BBF1000F07D0029088B94FF0FF347E
:105290000648784416301AE05FEA000A08D103484D
:1052A000784408304FF0FF34283010E000720000DE
:1052B000287FA8B9E87F98B1696851F8040B696044
:1052C000B0F1004FC0F007804FF0FF3471A000F044
:1052D00091F9201AD6E0A969884288BF0846A861DA
:1052E00009940A9606974FF0FF38039ECDF820B038
:1052F0000024DDF808B007E00AF8017B0120A96965
:10530000A877491EA9610226E8682969401C491E40
:1053100000292961E86024D4286801220021C847B7
:10532000074617F1010F1ED148462C46DDF80490C0
:10533000089D3A462146FFF751F9B9F1000F03D015
:10534000F0B2022800F08F80F0B2022800F09980BD
:10535000F00703D417F1010F40F089804FF0FF30C0
:1053600090E04746E0E70198002803DD384600F06A
:1053700076FB10E01FD50A98002809980ED1002866
:10538000009A0698394604D100F070F90028CBD075
:1053900011E000F06BF90028C6D10CE00028009A5B
:1053A0000698394603D1FFF701FF20B9BCE7FFF7A4
:1053B000FDFE0028B8D1089838B9287F0028A2D16E
:1053C000A869002898D10126AEE703A801460790F6
:1053D0000F55641C04AB224602A800F0F0F8811CB3
:1053E00002291BD8DFE801F002061400042C46F065
:1053F000010689D3002C07DD0798641E2946025D4B
:105400004846FFF7EBF8F5E7F6B286BB404639E0D1
:10541000029919B903A800F00DF9401C10F1030F0F
:1054200008BF0020064608E00798EA68641E521E7E
:10543000015DEA6000222868C847A642F4DB287FA5
:1054400058B9A86908B901265EE702984BF8040B21
:105450000121A869A977401EA86102266869401E3B
:105460006861002450E7207F58B9A06908B900207E
:1054700008E0002D19BF0020CBF8000000218AF8B9
:10548000001001200BB0BDE8F08F00000000F07F9D
:10549000FEFFFF7F7363616E665F733A2062616433
:1054A0002025632C2025732C206F7220255B207310
:1054B000697A65007363616E665F733A2062616446
:1054C00020696E746567657220617267756D656EBF
:1054D00074000000613807E005E0A0F161011A29BD
:1054E00001D20120704741381A288041C00F70470F
:1054F000A0F10901052901D3202801D1012070471D
:1055000000207047A0F141011A2938BF20307047B0
:105510003048704770B45368D41801E05B1C491ED2
:10552000042B08DA00291FBF057804F8015B10F886
:10553000016B002EF2D1536070BC704738B5144631
:105540001D4661B1FFF7E6FF61686A6B2046904730
:105550006FF00102811A02D0491E01D001E024E05F
:1055600026E00021616032BD38B5044608461100CE
:105570001D4615D02A46FFF7CDFF6968049B1CB96C
:105580005A6B2846904704E00A469B6B2946204602
:1055900098476FF00102811A02D0491E01D001E044
:1055A00003E005E00021696032BD6FF0010032BD0B
:1055B0004FF0FF3032BDDA6B1047064BBEE71CB52B
:1055C000044C0094FFF7D0FF16BD024BF3E70248EE
:1055D00070470000B801002080010020C9B20278A5
:1055E0008A421AB11CBF10F8012FF9E718BF00203A
:1055F0007047000080B500B906A005490B681BB1D3
:1056000022220021984701E0FCF756F8222002BD33
:1056100038090020636F6E73747261696E7420685C
:10562000616E646C65723A20626164206D657373AB
:105630006167650000F10103810704D010F8011BC8
:10564000820781B1FAD10268A2F10131914311F0D0
:10565000803104BF50F8042FF6E709BAB1FA81F19E
:1056600000EBD100401CC01A70470000C9B283078C
:1056700006D0521E22D310F8013B9942F7D11FE009
:10568000083A13D302F1040241EA012141EA01413F
:1056900050F8043B121F21BF4B40A3F1013C2CEA00
:1056A000030C1CF0803FF3D0C9B2001F083210F881
:1056B000013B521E28BF91EA030FF8D818BF012002
:1056C000401E70474AB1000011F8013B521E00F81D
:1056D000013B1CBF11F8013BF8E7704710B51446B9
:1056E00000F002F8226010BDC1F30A5343B14A0032
:1056F00012F5001F28D2A3F2FE32A1EB025170472F
:1057000050EA410C20D001F0004C31EA0C01B1FA12
:1057100081F204BFB0FA80F3D2180B3AB2F1200341
:105720002CBF00FA03F1914041EA0C013EBFC2F1E7
:10573000200C20FA0CF319439040524240F2FD3302
:10574000D21A01EB03517047002270474FF4001C3E
:105750001CEB410F94BF1CEB430F09E041EA030C23
:1057600050EA4C0C52EA0C0C03D2994208BF90420A
:10577000704714BF8B428242704700004FF4001CF8
:105780001CEB410F94BF1CEB430F09E041EA030CF3
:1057900050EA4C0C52EA0C0C03D28B4208BF8242F6
:1057A000704714BF9942904270470000124254D48F
:1057B00040F2FF7C1CEA11530FD0634531D09B1897
:1057C00063453CBF01EB0251704701F0004141EAE3
:1057D0000C510020AFF30080704750EA410320D005
:1057E00001F0004C91EA0C011CD0B1FA81F30B3BA3
:1057F0009A420DD9D21A994051EA0C01C3F1200CFA
:1058000020FA0CFC61449840531C40F2FF7CD7E71F
:10581000914041EA0C01C2F1200C20FA0CF319432B
:1058200090407047B0FA80F31533202BE0D3202A44
:10583000EED3203A203B9A4209D9D21A00FA03F15A
:1058400041EA0C010020531C40F2FF7CB8E700FA4B
:1058500002F141EA0C0100207047524240F2FF7C05
:105860001CEA11530DD06345DBD0B2EB030C3CBFF7
:10587000A1EB025170470CF1010221EA035141F4FE
:10588000801150EA410CCCD001F0004C352A27DCC5
:1058900030B481EA0C01B2F1200309DAC2F120032D
:1058A000044601FA03F5D0402843D1409C400CE067
:1058B000C3F12002450020FA03F418BF44F00104AC
:1058C00021FA03F091400C43002174F1004550F19E
:1058D000000051EB0C01244230BC7FF47BAF7047D9
:1058E0006146002076E70000C1F30A5340F2FE3221
:1058F0009B1A14DDD3F120034FEAE17208DDC902DF
:1059000041EA505141F00040D84080185040704763
:1059100003F2E13010B1D24382F000407047002022
:1059200070470000400D491840EA81200CD2490D13
:10593000A1F58061491C40F0004005DBD1F11F0159
:1059400054BFC840C01770470020704780B5FFF7AC
:10595000DFFD006C02BD0000D3BBD9B1B2F5803FC2
:105960005BD2022A1ED98C46B1FBF2F102FB11C3B5
:105970001B0443EA1043B3FBF2FC02FB1C3380B26E
:1059800040EA0343B3FBF2F002FB103240EA0C4062
:1059900000237047022A05D98446B0FBF2F002FBCF
:1059A00010C270474AB105D100F0010249085FEA10
:1059B0003000704700220023704700F029BC0B0024
:1059C0000200002100207047F7D300220023704717
:1059D000904271EB030CF2D370B5B1FA81F4B3FAD3
:1059E00083F52C1BA340C4F1200532FA05F633439E
:1059F000A2405FF00046E64002E05B085FEA320248
:105A0000841A71EB030524BF204629467641F4D35E
:105A100002000B003000002170BD70B5B1FA81F4B6
:105A2000B2FA82F5C4F120046419B4F12006DAD385
:105A3000B2405FF00044F440002502E052085FEA03
:105A40003303C61A71EB020E24BF3046714664411F
:105A50006D41F3D302000B002000290070BD10B58A
:105A60000446FFF755FD01462046096ABDE810408F
:105A7000084718B5044614F1010F83B00BD0082273
:105A8000002101A800F0C5FB01AA21466846FFF7E6
:105A90009CFD012803D04FF0FF3004B010BD9DF8ED
:105AA000000004B010BD10B50446FFF731FD0146FB
:105AB00020460969BDE81040084700002DE9B04CB8
:105AC00041EC100B2DED028B43EC182B53EC102BFB
:105AD00023F00041B1F5801F82B00DD200220029D1
:105AE00008BF0028009216D06A4651EC100BFFF751
:105AF000F5FD41EC100B0EE0DFF87444DFF878742C
:105B000004EB115000903B40DFF86804924643EAF2
:105B1000000B4BEC10AB53EC102B51EC180BFDF7BA
:105B200099F941EC100B0A465000009B400D1B18E0
:105B3000D0B1002B18DD40F2FF7083420CDB9FEDEB
:105B4000A20B53EC102B01F00041194355EC104B04
:105B50000D4645EC104B15E06FF31E5242EA03521E
:105B600051EC100B11460BE051EC100B20F0000231
:105B700031F0004308BF002A04D0009AFFF716FE58
:105B800041EC100B02B051EC100BBDEC028BBDE8E8
:105B9000B08C00002DE9F8452DED048B002A82B071
:105BA00041EC180B1D4600F0068157EC186B37F0DE
:105BB000004308BF002800F0FE8048004015401C4C
:105BC00002D1090300F0F780002A9FED819B40F18C
:105BD00095805242DFF8ECA1FA440AF5F47A4FF0CE
:105BE000080814460EE0E00707D5DAE9002351EC77
:105BF000190BFDF72FF941EC190B64080AF1080A9B
:105C0000A8F10108002C18BFB8F1000FEBD127F064
:105C10000041B1F5801F07D2002000906A4651EC88
:105C2000180BFFF75BFD0BE0DFF8442302EB11508C
:105C30000090DFF84013DFF8400307403046394357
:105C400053EC192BFDF7A4FA41EC180B0A4650004F
:105C5000009B400D1B18D0B1002B18DD40F2FF70E7
:105C600083420CDB9FED580B53EC102B01F00041ED
:105C7000194357EC106B0F4647EC186B15E06FF3A8
:105C80001E5242EA035251EC180B11460BE051EC44
:105C9000180B20F0000231F0004308BF002A04D0A6
:105CA000009AFFF783FD41EC180B51EC180B20F024
:105CB000000231F0004308BF002A66D048004015BA
:105CC000401C01D1090360D0002C5ED0AB4AAC4B24
:105CD00051EC180BFFF7F2FE20F0000231F0004308
:105CE00008BF002A41EC180B4FD048004015401C5B
:105CF00001D1090349D0641EE8D146E045DD314FAA
:105D00007F4407F1C00708261446E00707D5D7E906
:105D1000002351EC190BFDF79DF841EC190B6410B1
:105D20000837761E002C01DD002EEED153EC192B26
:105D300051EC180BFFF7C2FE20F0000231F00043D7
:105D400008BF002A41EC180B1FD048004015401C2A
:105D500001D1090319D0002C17DD8A4A924B51EC6E
:105D6000180BFFF7ABFE20F0000231F0004308BF34
:105D7000002A41EC180B08D048004015401C01D106
:105D8000090302D0641E002CE7DC51EC180B20F054
:105D9000000231F0004308BF002A05D0480040153A
:105DA000401C08D1090306D1AFF300801DB128685B
:105DB00040F00100286002B051EC180BBDEC048BE0
:105DC000BDE8F48564670000000000000000F07F7B
:105DD000000000000000F03F2DE9F14D81B05FEAC6
:105DE00003082DED028B84B01CBF0020C8F8000012
:105DF000079D0C46934607A800F015FAC11020F045
:105E00000800012801F0010A30D10220009001AB06
:105E100007992246284600F097FA040008BF9FED34
:105E2000630B1ED00298FDF703F8022C41EC100B17
:105E300017DB03AF661E9FED548B51EC100B53EC38
:105E4000182BFDF707F8044657F8040B0D46FCF72E
:105E5000EFFF22462B46FDF7DDF8761E41EC100BD6
:105E6000EBD10198434600EB0B025FE0022864D1BE
:105E7000009001AB07992246284600F041FB040040
:105E800008BF9FED4A0B1ED00298FCF7D1FF022CF1
:105E900041EC100B17DB03AF661E9FED3D8B51EC01
:105EA000100B53EC182BFCF7D5FF044657F8040BE6
:105EB0000D46FCF7BDFF22462B46FDF7ABF8761EDC
:105EC00041EC100BEBD151EC100B0B46019A580032
:105ED000400D02EB00041AD0002C18DD40F2FF70D8
:105EE00084420CDB9FED2C0B53EC102B01F0004196
:105EF000194355EC104B0D4645EC104B14E06FF375
:105F00001E5343EA045351EC100B19460AE051ECBE
:105F1000100B20F0000431F0004508BF002C03D026
:105F2000FFF744FC41EC100B43465A4651EC100B72
:105F3000FFF730FE41EC100B0AE0032808BF9FED8D
:105F4000160B05D004280CBF9FED150B9FED170B0A
:105F5000BAF1000F05D051EC100B81F0004141EC7B
:105F6000100B04B051EC100BBDEC028BBDE8FC8DA6
:105F700002FCFFFF0000E03FFFFF0F80436FAC64B7
:105F80002806C80A3CBF737F0000000065CDCD41E4
:105F9000000000000000B041000000000000F07FA1
:105FA000FFFFFFFFFFFFFF7FDD4F157500000000C3
:105FB000000000002DE9FC4F85B00C4693460BB164
:105FC00000221A600290824601E00AF1010A9AF862
:105FD0000000FFF744FD0028F7D19AF800002D28B3
:105FE00018BF2B2807BF1AF8010B8DF800002B21D2
:105FF0008DF80010BBF1000F019405D4BBF1010F27
:1060000002D0BBF1250F04DB002C71D00298206078
:106010006EE0BBF1000F0DDDBBF1100F04BF9AF86D
:106020000000302802BF9AF8010040F020007828D4
:1060300014D10EE09AF80000302818BF4FF00A0B78
:106040000CD19AF8010040F02000782804D14FF0DC
:10605000100B0AF1020A01E04FF0080BCDF810A076
:1060600001E00AF1010A9AF800003028F9D0094845
:10607000784420300024283000260027CDF80CA0DA
:106080000025A0468DF80100DFF80890F94409F1D9
:10609000040918E0C86300009DF80110401A5FFA77
:1060A00080F85846A0FB06234FEAEB7100FB07334C
:1060B00001FB0633344600213D4612EB080643EB54
:1060C00001070AF1010A9AF8000000F01DFB0146E1
:1060D0005A4609F12800FFF7C9FA0028DCD10499D3
:1060E00051455A4607D1019810B1019902980860AC
:1060F0000020002130E0039919F80200AAEB010109
:10610000081A00281BD410DC0023B6EB080067EB4C
:1061100003018F4209D301D8864206D3D317FFF774
:106120001BFCA94208BFA04209D0AFF3008006982B
:1061300008B1012101604FF0FF36374606E09DF8B7
:1061400000002D2802D1764267EB4707019808B17D
:10615000C0F800A03046394607B0BDE8F08F000017
:1061600000BF002326E700002DE9F8430D0080461C
:1061700091461E4608BF6D46444600E0641C2078E8
:10618000FFF76DFC0028F9D127782D2F18BF2B2F92
:1061900005D114F8010FFFF762FC50B900E02B277E
:1061A00033464A4629462046FFF704FF2A689442B0
:1061B00005D1C5F8008000200021BDE8F4832B2F15
:1061C00005D14FF00043994209D2BDE8F4832D2F49
:1061D000FBD1B1F1004F12D301D801280FD3AFF397
:1061E00000800EB1012030602D2F19BF4FF0FF301D
:1061F0006FF0004100204FF00041BDE8F4834042C1
:1062000061EB4101BDE8F48300BF0023ACE700006F
:10621000704710B5044610460A4601462046FBF773
:10622000A1FA204610BD2DE9F84305460C462E681C
:10623000002700E0761C3078FFF711FC0028F9D128
:1062400030782D280CBF08272B2800D1761C3078F9
:1062500040F020016E2927D1707840F0200061289D
:1062600002BFB07840F020006E2802D02E680027D0
:1062700046E0F61CB046042798F8000028283FD1D5
:1062800018F8019F4846FFF70EFC0028F8D1A9F145
:1062900030000A28F4D398F800005F28F0D02928AD
:1062A0002ED108F101062BE069292CD1707840F03D
:1062B00020006E2802BFB07840F02000662802D08F
:1062C0002E6800271CE016F8030F40F02000692814
:1062D00002BF707840F020006E2847F003070FD10E
:1062E000B07840F02000692802BFF07840F020002C
:1062F000742805D1307940F02000792808BF761D38
:10630000F4B126601CE0302802BF707840F0200015
:10631000782813D1B01C01782E2908BF401C0078C2
:10632000A0F16101062921BFA0F14102062A3038FF
:106330000A2803D2B61C47F0020701E047F0010724
:106340002E603846BDE8F2832DE9F14F8CB04FF056
:106350000008169DC34605EBC5052D2DC3F800B0FA
:106360009246C8BF2D25C3F804B0D94602E0491CA7
:106370004FF0010908783028F9D0002411E018689E
:10638000401C18600A78302A08D04FF0010805E058
:10639000AC42F4DA30380DF80400641C491C4FF0AC
:1063A00001090878A0F130020A2AF1D30F461E46EF
:1063B000FFF70DF9406A39780278914208BF7F1CD7
:1063C000002C48460ED1397830290BD13068401E58
:1063D00030607F1C0120F6E7302918BF4FF001081C
:1063E0007F1C01203978A1F130020A2A0AD2AC427E
:1063F000F2DAA1F130000DF80400641C3268521E7C
:106400003260EDE7B8F1000F0DD00DF1FF314A5DBC
:10641000521C4A5507E00DF1FF32115D49B932684F
:10642000521C3260641E002CF5DC04BF8DF800B0F5
:106430000124002857D04FF0090994FBF9F9C4F161
:10644000090309EBC9010B44092193FBF1F1002277
:1064500001EBC101591A1AD04FF0010B17E056F8A1
:106460002B1001EB810105EB410146F82B100CE0EC
:10647000092193FBF1F101EBC1011DF80250591AFA
:10648000EDD10BF1010B46F82B505B1C521CA242C4
:10649000EEDB397841F02001652924D1394617F81F
:1064A000012F164D2B2A16BF2D2A17F8014B2B242E
:1064B0000022002308E0AB4204DA03EB83020CEB7A
:1064C0004203303B7F1C012297F800C0ACF1300E34
:1064D000BEF10A0FEFD32D2C346808BF5B421B19A5
:1064E000336002B90F46BAF1000F03D000B90C9F18
:1064F000CAF8007058460DB0BDE8F08F00E1F50510
:106500002DE9F14F8CB04FF0000ADDF85880C3F848
:1065100000A0C8EBC808B8F1230FC8BF4FF023088C
:106520009146C3F804A0002701E0491C0127087820
:106530003028FAD068A201925FF000046CA20092A9
:106540000DF1080B0D461E460EE03068401C306011
:1065500008E0A045F9DB019A0099801A085C0BF865
:106560000400641C6D1C012795F800105AA0162227
:10657000FFF77CF80028ECD1FFF729F8406A29786A
:106580000278914208BF6D1CB4B92878302813D125
:106590003168491E31606D1C0127F6E7A04509DB13
:1065A000019A0099801A085C0BF80400641C316899
:1065B000491E31606D1C01272978162246A0FFF77D
:1065C00055F80028EAD1A04517DA1BF8081007296A
:1065D00006DD0DF1070111F80820521C01F8082012
:1065E00044463268521C326007E00DF10702115D2B
:1065F00049B93268521C3260641E002CF5DC04BFBD
:106600008DF808A0012431688900002F316055D031
:106610004FF0070C94FBFCFCC4F10703CCEBCC0C53
:106620006344072193FBF1F10022C1EBC101591A28
:1066300018D04FF0010A15E056F82A100CEB0110A3
:1066400046F82A000CE0072193FBF1F1C1EBC101F0
:106650001BF802C0591AEFD10AF1010A46F82AC004
:106660005B1C521CA242EEDB297841F0200170290C
:1066700024D1294615F8012F16482B2A16BF2D2A9A
:1066800015F8014B2B240022002308E0834204DA92
:1066900003EB83020CEB4203303B6D1C012295F8A7
:1066A00000C0ACF1300EBEF10A0FEFD32D2C3468D0
:1066B00008BF5B421B19336002B90D46B9F1000FE8
:1066C00003D007B90C9DC9F8005050460DB0BDE885
:1066D000F08F000000E1F5053031323334353637C4
:1066E000383961626364656641424344454600004F
:1066F000000102030405060708090A0B0C0D0E0F22
:106700000A0B0C0D0E0F000010B50446FEF700FF3B
:1067100001462046896ABDE81040084738B500F0B8
:1067200023F800F0C8FB00F019F800F0C8FB31BDF9
:1067300038B500F019F800F0BEFB00F00FF800F0DB
:10674000BEFB00F005FA00F037F800F006FA00236F
:10675000042229462046FBF795F824E00220009009
:106760000423DFF8B429704704460D4600200CE0EE
:106770004FF4A6714143401C6A5C42F001026A5426
:1067800029444B7B03F03F034B73A042F0DB2046D0
:1067900000F0D8BD38B500F0E4F900F0D9F900F008
:1067A0000BF800F0DAF92946204601B0BDE8304088
:1067B00000230422FBF7E4B8022000900423DFF852
:1067C0005C29704710B500F04FF800F066F8DFF86C
:1067D0005049E278A178207800F0D6FD00F059F811
:1067E00060600FF6D01024E010B500F03DF800F026
:1067F00054F8DFF82C09C2780078012100F0C4FDBC
:10680000082000F065FDBDE810400FF6A810FCF769
:1068100032B810B500F028F800F03FF8DFF8004972
:10682000E178A07800F0BCFD00F033F860600FF66E
:10683000A010FCF720F86068BDE81040FCF720B815
:1068400010B500F011F800F028F8DFF8D408C1788E
:10685000012000F0A5FD082000F03AFDBDE8104041
:106860000FF66C10FCF707B8044600F04ABC10B5F0
:10687000FFF7FAFF00F011F8DFF8A448E278A178FA
:10688000012000F081FD00F004F86060DFF894085A
:10689000CFE7DFF8940801F0F4BD204600F052BDC8
:1068A00010B5FFF7E1FFFFF7F8FFDFF87408C278D3
:1068B0000121012000F068FD082000F009FDBDE87D
:1068C0001040DFF86008FBF7D6BF38B500F049F993
:1068D00000F0B8F800F041F900F0AEF800F03DF932
:1068E00000F0A4F800F039F929462046FBF74AFAEF
:1068F00029462046FBF73AFB29462046BDE83440AE
:10690000FBF775BB38B504460D46002001E000F0EA
:1069100041FBA042FBDBFFF7C0FF00F0CCFA00F028
:106920007FF800F01AF929462046BDE83440FBF70D
:106930009BBC38B500F015F900F06CF800F00DF9CB
:1069400000F062F800F009F90A2000900B23DFF84C
:10695000DC2700F002F929462046FBF743FC2946D4
:106960002046FBF791FB29462046BDE83440FBF763
:10697000F7BB7CB500F0F5F800F064F800F0EDF836
:1069800000F05AF800F0E9F800F050F800F0E5F8EF
:1069900000F046F800F0E1F800F03CF800F0DDF817
:1069A00000F032F800F0D9F80A2000900B23DFF84D
:1069B0007C67324600F0D1F80A2000900B23324663
:1069C00000F0CBF829462046FBF7DCF929462046A3
:1069D000FBF7CCFA29462046FBF709FB294620465F
:1069E000FBF742FC29462046FBF7FCFB29462046E4
:1069F000FBF74AFB29462046FBF7B2FB2946204617
:106A0000BDE87C40FBF7ACBB0A2000900A23DFF80E
:106A1000202770470A2000900923DFF818277047C5
:106A20000A2000900823DFF8102770470A20009002
:106A30000723DFF8082770470A2000900623DFF8B5
:106A4000002770470A2000900523DFF8F8267047DA
:106A500010B5DFF8CC4600F075FCE078092100F0B5
:106A6000A7FCFFF716FF60600FF28070E1E638B513
:106A700000F077F800F066F800F06FF800F056F8D4
:106A800000F06BF800F046F800F067F800F03CF812
:106A900000F063F829462046BDE838400022FBF7A5
:106AA000A9B938B500F05DF800F046F800F055F8E7
:106AB00000F036F800F051F81FE038B500F051F85A
:106AC00000F040F800F049F800F030F800F045F828
:106AD00000F020F800F041F800F016F800F03DF862
:106AE00000F02AF800F039F800F01AF800F035F854
:106AF000002229462046FBF77DF929462046BDE8BD
:106B000038400222FBF776B9042000900023DFF81A
:106B100038267047032000900023DFF830267047A6
:106B2000022000900223DFF8282670470220009000
:106B30000023DFF820267047012000900223DFF8B1
:106B400018267047012000900023DFF810267047B8
:106B5000012000900423DFF808262946204601F092
:106B600005BB04460D4600F0EDBB38B5FFF7F9FF55
:106B7000072000900123DFF8EC25FFF7EEFF082047
:106B800000900123DFF8E025FFF7E7FF29462046C4
:106B9000BDE838400122FBF72DB910B500F0D2FB5B
:106BA000DFF87C45607800F012FCFFF772FE606051
:106BB0000FF254603DE638B5FFF7D3FF00F043F81D
:106BC000FFF7CBFF2946204601B0BDE83040012346
:106BD0000CE038B5FFF7C5FF00F02FF8FFF7BDFF59
:106BE0002946204601B0BDE8304003230C22FBF7C4
:106BF0008DBB38B5FFF7B5FF00F025F8FFF7ADFF07
:106C0000022000900C23DFF86425FFF7A6FF00F0B8
:106C100014F8FFF7A2FF042000900C23DFF85025A2
:106C2000FFF79BFF00F00BF9FFF797FF294620467F
:106C300001B0BDE830400023D8E7032000900C23CA
:106C4000DFF830257047012000900C23DFF828255D
:106C5000704738B5FFF785FF0A2000900F23DFF853
:106C60001C25FFF77AFF29462046BDE838400F2251
:106C7000FAF720BF80B500F065FBDFF8040501F0EE
:106C80007CF9BDE802400FF29C50FBF7F4BD80B5E3
:106C900000F058FBDFF8EC0401F06FF9BDE80240AA
:106CA0000FF29050FBF7E7BD80B500F04BFBDFF82B
:106CB000D80401F062F9BDE802400FF29450FBF7EE
:106CC000DABD80B500F03EFBDFF8C00401F055F9F5
:106CD000BDE802400FF28450FBF7CDBD2DE9FE4F19
:106CE00080460D460FF280500FF2B4540FF2A459B3
:106CF0000FF2945ADFF898B4FBF7BDFD02A8FBF73A
:106D0000D7FD404600F01EFB002753E0022851D17A
:106D100039460BF12800FCF71FF85046FCF71CF829
:106D20004846FCF719F82046FCF716F80FF27C509D
:106D3000FCF712F80FF28050FCF70EF80FF28450B7
:106D4000FCF70AF801A992A0FCF746FB002129E014
:106D50004FF4A67078432E18295C41F001012954A4
:106D60007F1C02980128D1D139465846FBF7F4FF21
:106D70005046FBF7F1FF4846FBF7EEFF2046FBF7D6
:106D8000EBFF0FF22850FBF7E7FF0FF22C50FBF759
:106D9000E3FF0FF23050FBF7DFFF01A97CA0FCF707
:106DA0001BFB01210198C0B200F027FB317960F391
:106DB0000501317140468742CADB00F0C3FA012069
:106DC00000900423DFF8CC232946404601F0D3FA93
:106DD00000F092F92946404601F0C8F900F02FF87A
:106DE0002946404601F0C2F90123042229464046C3
:106DF000FAF748FD0123042229464046FAF7C0FD70
:106E000005230C2229464046FBF780FABDE8F78FA0
:106E10007CB500F058F800F04EF8FFF799FE00F04E
:106E20000EF8FFF79AFE00F0AEF800F048F800F018
:106E3000D8FA00F0A3F8FFF790FED7481AE0052033
:106E400000900C23D54A70477CB500F03CF800F068
:106E500032F8FFF77DFEFFF7F2FFFFF77EFE00F04E
:106E600092F800F02CF800F0BCFA00F087F8FFF779
:106E700074FECB48FBF7FFFC012304222946204681
:106E8000FAF700FD0123042229462046FAF778FD8F
:106E900005230C2229462046FBF738FA0E22294604
:106EA0002046FAF759FE2946204602B0BDE8704058
:106EB0000E22FAF7ABBE012000900423B54A294602
:106EC000204601F058BA04460D46002008261CE072
:106ED0004FF4A6714143401C6A5C42F001026A54BF
:106EE00029440922CB7843F00F03CB708A31002369
:106EF0000B704A700F234B718A7055238B71AA2235
:106F0000FF23CE700E71CA710B72A042E0DB2046E7
:106F100000F018BA7CB504460D460020002615E0A6
:106F200000F038F829440622CB7843F00F03CB70E9
:106F30008A3108230B704B70CA70A0238B71092211
:106F400025230E714E718A70CE710B72A042E7DB61
:106F5000FFF7A3FCFFF7AFFFFFF7FAFDFFF76FFFA7
:106F6000FFF7FBFD00F00FF8FFF7A9FF00F039FA7B
:106F700000F004F8FFF7F1FD8A487BE70A20009053
:106F80000E23894A70470A2000900E23874A7047D3
:106F9000256400004FF4A6714143401C6A5C42F036
:106FA00001026A5470472DE9FC42054600224FF465
:106FB000A6770C4600261BE007FB02F0521C215C62
:106FC00041F00101215420440621C37843F00F030E
:106FD000C3708A300823C1700370067106234371A1
:106FE0000821A023417081708371C671A1230372AF
:106FF000AA42E1DB284600F0A5F901200090042315
:10700000644E00F06FF800F077F800F071F805209A
:1070100000900C23DFF8849100F069F8FFF7B3FFCC
:1070200000F061F800F0DDF9012304222146284632
:10703000FAF728FC0123042221462846FAF7A0FC8F
:107040000E2221462846FAF787FD05230C22214609
:107050002846FBF75BF90022FF211FE007FB02F047
:107060004FF0090C235C43F00103235420444FF0FC
:10707000070EC37843F00F03C3708A300023C37038
:1070800080F800C080F804E080F801C080F805E0D6
:1070900080F802C08171C1710172521CAA42DDDB0D
:1070A000284600F04FF901200090042300F01AF860
:1070B000052000900C2300F01AF800F092F9FFF779
:1070C0005DFF00F015F83A48FBF7D5FB0E2221468C
:1070D0002846FAF79BFD2146284602B0BDE8F0425B
:1070E000052383E532462146284601F044B94A4645
:1070F0002146284601F03AB8012000900423184A9E
:10710000704780B500F01EF91D4800F036FFBDE85D
:107110000240082000F0DCB8020300200603002033
:1071200030090020F4C600082C03002018030020BA
:107130001603002014030020120300200C0300207B
:107140000A03002008030020200300201E03002063
:107150001C030020100300201A0300200E0300204F
:10716000040300203C0300203E03002024030020F1
:1071700028030020260300202203002032030020E1
:107180003A03002034030020360300203803002097
:107190000CC400080003002018C700082A030020C0
:1071A0003CC7000804C60008300300202E0300205E
:1071B0002CC600084164693120636F6E7665727376
:1071C000696F6E20636F6D706C657465640000009C
:1071D0004164693220636F6E76657273696F6E20E9
:1071E000636F6D706C6574656400000041647620A7
:1071F000636F6E76657273696F6E20636F6D706C0E
:107200006574656400000000416461757820636FF7
:107210006E76657273696F6E20636F6D706C6574E6
:1072200065640000536F6674205265736574204472
:107230006F6E6500436F6D6D616E6420436F756E98
:1072400074657220526573657420446F6E6500002A
:10725000536E617020446F6E65000000556E736E52
:10726000617020446F6E6500506C656173652045E8
:107270006E7465723A200A313A5365740A323A5292
:10728000657365740A00000030203A2047504F3182
:10729000200A000031203A2047504F32200A0000D7
:1072A00032203A2047504F33200A000033203A2042
:1072B00047504F34200A000034203A2047504F35C1
:1072C000200A000035203A2047504F36200A00009F
:1072D00001F020B9002200E001224FF400412448CF
:1072E00001F00DBA0A460146224800684FF0FF330C
:1072F00001F06BBA70B50C461E4E0146154630685B
:107300004FF0FF33042201F060FA30682A4621462C
:10731000BDE8704003E00A460146164800684FF099
:10732000FF3301F0E5BA1448006801F0C6BD124809
:10733000006801F0D1BD104801680968486A002260
:107340004A62704770B504460025094E0CE00022E1
:1073500000F014F80120FFF7BBFF012200F00EF847
:10736000012001F0D7F86D1CE8B2A042EFD370BD48
:1073700000000240680100206C0100204FF4004131
:10738000304601F0BCB9000080B502F00302801C59
:1073900002EBC1128DF8000060328DF8012012E07E
:1073A00080B501F0030101EBC0110122683106E054
:1073B00080B501F00F0101EBC011042230318DF8CE
:1073C00000208DF80110684600F0D7FD01BD80B5A2
:1073D00000F00300303005218DF801008DF8001019
:1073E000F1E780B5FFF776FF0D21DFF8D004FFF756
:1073F00079FFBDE80140FFF76FBF01290CBF01FA1B
:1074000000F00020C0B27047F0B5002500268FE0E4
:1074100000F0F2F803F1A8042F6827606F68676036
:10742000751C277893F806C007F001070CF0F70CDD
:107430004CEAC70C83F806C00CF0F90C2778C7F3A8
:1074400041074CEA470C83F806C00CF0FE0C277885
:107450004CEAD7179F71ED00677893F808C0DF7189
:107460000CF0F80CA778C7F3C20747EA0C071F72A5
:10747000761CA77893F808C0C7F380170CF0F70CB8
:107480004CEAC70C83F808C00CF0EF0CA778FF0992
:107490004CEA07171F72E77893F809C007F01E0738
:1074A00067F3030C83F809C0E77894F804E04FEA27
:1074B000171C4FEA0E1E0CF00E0C0EF0300E4EEAAA
:1074C0000C0C07F0010747EA0C0793F80AC00CF010
:1074D000C00C47EA0C079F7293F80AC06779C7F39C
:1074E000401700F064FB83F80AC00CF07F0C67794A
:1074F000FF084CEAC7179F7293F80BC06779C7F370
:1075000080070CF0FE0C47EA0C07DF7293F80BC003
:107510006779C7F340070CF0FD0C4CEA4707DF72B0
:1075200007F0FB07647904F0010447EA8404DC7285
:107530008642FFF66DAFF0BDF0B50025002658E09D
:1075400000F05AF803F1B6042F6827604FF6807EEA
:107550006F686760751C2778B3F810C007F07F0765
:107560000EEA0C0C47EA0C071F824CF27F0E2778BC
:1075700093F811C0FF097F000CF03F0C4CEA87170D
:107580005F74ED006778B3F810C007F07F070EEA6C
:107590000C0C4CEAC7171F82761C677893F811C051
:1075A000FF090CF03F0C4CEA87175F7493F812C088
:1075B000A77807F007070CF0F80C47EA0C079F7450
:1075C00093F812C0A778C7F3C2070CF0C70C4CEAB7
:1075D000C70C83F812C00CF07F0CA778BF094CEAE7
:1075E000C7179F7407F0BF07A478E40947EA84141B
:1075F0009C748642A4DBF0BD4FF4A673EDB27343D6
:1076000015440B447047012A02D0022A02D0704769
:107610001A46F9E61A468FE7F0B5002600230BE07C
:1076200000F06CF807EB0C2EAF780EEB0747A76164
:1076300000F088F8E5615B1C8342F1DBF0BDF0B53A
:10764000002500231BE04FF4A674EDB25C43154403
:107650000C4404F1D2062F6837606F68776004F13C
:10766000D406377896F801C007EB0C2727855D1CF8
:10767000B778F67807EB0626ED0066855B1C83423B
:10768000E1DBF0BDF0B5002600230EE000F036F897
:1076900007EB0C2EAF780EEB07476763F6002F79E8
:1076A0006D7907EB052525875B1C8342EEDBF0BD7A
:1076B000F0B5002400230BE000F099F905F1D206A3
:1076C00000F08EF905F8747FE40076786E705B1C2C
:1076D0008342F1DBF0BDF0B5002600230BE000F0A3
:1076E0000DF807EB0C2EAF780EEB0747276200F082
:1076F00029F865625B1C8342F1DBF0BD4FF4A67490
:10770000F6B25C4316440C4404F1D20537682F608E
:10771000776895F801C06F605E1C2F787047F0B5F0
:10772000002600230BE0FFF7E9FF07EB0C2EAF78F4
:107730000EEB0747E76200F005F825635B1C834208
:10774000F1DBF0BDF600EF7895F804C06D7907EB3A
:107750000C2707EB05457047F0B5002600230BE02A
:10776000FFF7CCFF07EB0C2EAF780EEB0747E76374
:10777000FFF7E8FF25645B1C8342F1DBF0BD0000EE
:107780002DE9F04700F0EBF80CBF1824082400F0B6
:10779000A8F8070001D14A485FE000212FE000F07F
:1077A000C2F800F056F87B7B3A7B02EB0322828121
:1077B000FB7BBA7B02EB0322C2817B7C3A7C02EB2F
:1077C00003220282FB7CBA7C02EB032242827B7D95
:1077D0003A7D02EB03228282FB7DBA7D0BE03A7890
:1077E0007B7802EB03224282FB78BA7802EB032219
:1077F00082827B793A7902EB0322C282761C46456B
:1078000026DA00F068F800F05FF84430042DF5D86F
:10781000DFE805F00506090E0400EFE7DFE7BEE745
:1078200000F064F8EAE700F071F800F012F8E5E71C
:107830003A787B7802EB03228281FB78BA7802EBFC
:107840000322C2817B793A7902EB03220282D5E7D7
:107850002FE002EB032242817047FBF70CF8002077
:1078600001F0F6FD00BF2DE9F04700F078F80CBFFD
:107870000C24082400F035F8070001D11148ECE78A
:10788000002107E000F04FF801E000F03FF8FFF7BB
:10789000E0FF761C46450CDA00F01DF800F014F805
:1078A0006830002DEED0022DEFD0F2D200F01EF89D
:1078B000EFE73846BDE8F04701F0CCBD00000020FE
:1078C00060C7000854C600084FF4A6707043711CCE
:1078D000484461437047C9B2224651443846FDF7D7
:1078E000F1BE9A4601212046F9F7C4BE3B787A786A
:1078F00003EB02220280BB78FA7803EB022242807B
:107900007B793A7902EB0322828070473A787B7860
:1079100002EB0322C280FB78BA7802EB03220281D9
:107920007B793A7970473A787B7802EB03220280C0
:10793000FB78BA7802EB032242807B793A7902EB3A
:1079400003228280FB79BA7902EB0322C2807B7A20
:107950003A7A02EB03220281FB7ABA7A7047154623
:107960000026002D804689467047F0B5002500238B
:107970001CE000F0C8F906F1E0042F6827606F688A
:1079800094F801C067605D1C277847EA0C2726F849
:10799000767FED00A77894F803C047EA0C2777803C
:1079A0005B1C2779647947EA0427B7808342E0DBD0
:1079B000F0BDF0B5002400230FE000F018F805F149
:1079C000EE0600F00DF805F87C7FE40077786F7024
:1079D0005B1CB778AF70F678EE708342EDDBF0BDDC
:1079E00027683760676877605C1C377870474FF4AA
:1079F000A675E4B25D4314440D447047F0B500240D
:107A00000025C8E04FF4A673E4B26B431444CE18CB
:107A100006F1FC0327681F6067685F606C1C1F78B5
:107A200016F880CF07F001070CF0FE0C47EA0C07B0
:107A30003770E4001F7896F800C0C7F340070CF0D9
:107A4000FD0C4CEA470C86F800C00CF0FB0C5F788C
:107A500007F001074CEA870C86F800C00CF0F70C21
:107A60005F78C7F340074CEAC70737706D1C9F78F3
:107A700093F803C0B6F802E0BF0107F4F86747EADD
:107A80009C070EF4784E47EA0E07778096F800C000
:107A9000DF7807F003070CF0CF0C4CEA07173770BC
:107AA00096F804C01F7900F087F886F804C00CF03F
:107AB000FD0C1F79C7F340074CEA470C86F804C059
:107AC0000CF0FE0C1F79C7F3800747EA0C073771EB
:107AD00096F803C01F7900F062F8F77096F803C0BB
:107AE0001F7900F062F886F803C00CF0DF0C1F79F4
:107AF000C7F340174CEA471C86F803C00CF0EF0CA4
:107B00001F79C7F380174CEA071C86F803C00CF0F6
:107B1000F70C1F79FF094CEAC707F77096F805C004
:107B20005F7900F049F886F805C00CF0FD0C5F792C
:107B3000C7F340074CEA470C86F805C00CF0FE0C72
:107B40005F79C7F3800747EA0C07777196F804C09E
:107B50005F7900F024F8377196F804C05F7900F07F
:107B600024F886F804C00CF0DF0C5F79C7F34017E7
:107B70004CEA471C86F804C00CF0EF0C5F79C7F3A1
:107B800080174CEA0717377107F0F7075B79DB09B5
:107B900047EAC30333718542FFF634AFF0BDFF08F7
:107BA0000CF07F0C4CEAC7177047C7F300170CF0B6
:107BB000BF0C4CEA871C704707F001070CF0FB0C68
:107BC0004CEA870C7047F0B50023002412E04FF414
:107BD000A675DBB2654313440D4405F585761F6831
:107BE00037605F687760631C95F80F6185F8866081
:107BF000DB00641C8442EADBF0BDF0B50024002306
:107C000034E0FFF7F4FE05F58C7627683760676887
:107C1000776005F58E76377815F887CF07F01E0761
:107C200067F3030C85F800C05C1C377896F801C038
:107C30004FEA0C1C4FEA171E0CF0300C0EF00E0E23
:107C40004EEA0C0C07F0010747EA0C0795F801C053
:107C50000CF0C00C47EA0C076F70E400AF78767840
:107C600007F0F00747EA1616AE705B1C8342C8DBCC
:107C7000F0BD000010B51446641E042C1A4613D83B
:107C8000DFE804F00306090C0F00BDE810406CE6C5
:107C9000BDE810408DE6BDE81040AFE6BDE81040FD
:107CA00091E7BDE81040A8E710BDF0B5002500231E
:107CB00026E000F028F806F593742F6827609336C5
:107CC0006F6867605D1C27783F09F770ED002778C3
:107CD00007F00F0737705B1C6778B771A7783F090B
:107CE0003771E778F771A77807F00F077770277972
:107CF0003F09777167793772247904F00F04B47003
:107D00008342D6DBF0BD4FF4A674EDB25C4315445C
:107D10000E197047F0B50025002317E0FFF7F3FFB9
:107D200006F59A742F6827606F6867605D1C277876
:107D300006F89C7FED00677877705B1CA778B770BA
:107D4000E778F77027793771647974718342E5DBDE
:107D5000F0BDF0B500223BE000F09DF804F1A20375
:107D6000257805F0060646EAC516C5F3C0052E437C
:107D70001E70521C65785D70A5782E09ED0005F027
:107D8000780545EAC6159D70E77825792E017F00B4
:107D900006F0E00607F01E073E4305F001053543F7
:107DA000DD702579C5F301151D71657924796608A3
:107DB00006F02006E40946EAC406AC0004F0040418
:107DC000264305F002073E43C5F3800426435E7157
:107DD0008242C1DBF0BD70B5002221E04FF4A673F2
:107DE00053430B4403F1B0041D7B05F07F05257060
:107DF000521C9D895E7BED09B60905F07F0545EAB9
:107E0000C61565709B7BDE099D09B60146EAC5165D
:107E100003F03F033343A3700023E37023716371C6
:107E20008242DBDB70BDF0B5002231E000F033F8B8
:107E300004F1BE03257D05F003051D700026257D98
:107E40009E70C5F381055D70DE70521C667D257DD8
:107E5000F708360106F0700646EAC716EF0946EA4B
:107E6000C706C5F302152E431E71657DA47D67010B
:107E7000A60807F04007240147EAC61704F01004DB
:107E80003C43EE0944EAC604C5F302152C435C7179
:107E90008242CBDBF0BD4FF4A6735343CC1870473E
:107EA00070B5002220E0FFF7F6FF04F590738A34E6
:107EB000521C2678E57806F00F0646EA05161E7075
:107EC000A5795D706578267905F00F0545EA0615F8
:107ED0009D70E579DD70A578667905F00F0545EAB6
:107EE00006151D71247A5C718242DCDB70BD0000D6
:107EF000F0B5024610200023DFF860450BE0DEB24B
:107F000085B28F5D87EAD51707F0FF0734F8175061
:107F100085EA00205B1CDDB29542F0D34004000CE2
:107F2000F0BD70B50446102000250EE0D35C80EA59
:107F300083000823460000F400700128B4BF3046D7
:107F400086F08F005B1EF5D16D1CEBB28B42EDDB32
:107F5000012C0FD1515C890001F47C71484006214D
:107F6000420000F400700128ACBF82F08F00104680
:107F7000491EF5D1C0F3090070BD80B501788DF8B8
:107F80000010694642788DF801200220FFF7B0FF0B
:107F9000010A8DF802108DF80300FFF79BF9042108
:107FA0006846FFF79FF9FFF797F901BD2DE9F84FF4
:107FB00084B082469DF83C00019005461AFB05F509
:107FC0000C46EDB216461F4601212846F9F752FB32
:107FD000804601980121F9F74DFB8146B8F1000F69
:107FE00018BFB9F1000F4FF0000B02D1DFF8700499
:107FF000B6E021788DF80010694660788DF80100B0
:1080000000240220FFF774FF010A8DF803008DF8A9
:1080100002105046FFF796F9FFF75CF92A464146F1
:108020006846FFF767F9FFF757F9019D0296039736
:10803000AD1E0E9E2EE08B18521C18F80370C7540C
:10804000AA42F8DB02900198411808EB010010F8F1
:10805000021D8908315507784078019A3F0207F4DC
:10806000407707435FFA8BF008EB00014846FDF7C5
:1080700029FB9DF83C10601C10FB01FB4A46294679
:108080000120FFF74EFF0399874214BF0120002013
:108090000855641C544504DA019902980022614392
:1080A000CEE7404601F0D6F9484601F0D3F905B0D5
:1080B000BDE8F08F2DE9FE430546EF003F1D0C465D
:1080C000FFB2904601213846F9F7D4FA060002D1F2
:1080D000DFF8900344E020783070022061787170FE
:1080E00004243146FFF704FFF070010A2846B170FE
:1080F000062526E0A0F1010905FB09F1002215FB88
:1081000000F353FA82F34344521C13F8063C3355F0
:10811000641CD3B2062BE4B2F1DBC9B2062241449F
:108120006846FDF7CFFA6A4606210120FFF7F9FEFF
:10813000010A3155641CE2B2641CB054E4B25FFA27
:1081400089F00028D6D1FFF7C5F839463046FFF749
:10815000C9F8FFF7C1F8304601F07CF9BDE8F783B4
:10816000FAF789FB002001F073F900BF2DE9FE4FFB
:10817000DDF830B081465FEA0B008A4690461E4625
:1081800010D1122E1CBF132E142E01D1222402E076
:10819000152E02D11024274607E00FF23C30FAF7E3
:1081A0006AFB02E04FEAC90408270121A0B2F9F7EF
:1081B00061FA054601214846F9F75CFA04460121B7
:1081C0004846F9F757FA002C18BF0028029000D053
:1081D00015B900BFC8A0C3E702980090FFB241469E
:1081E000019723462A464846FFF7E0FE0F2E4FF43C
:1081F000A67700F2A680DFE806F014A420A4082CDD
:108200003844505C687480A48C9800F0ABF8FFF799
:10821000FAF90020484516DA00F09EF882F83D1180
:10822000F8E700F09FF8FFF7ABFA002048450ADABC
:1082300000F092F882F84511F8E700F093F8FFF7A4
:1082400012FB002048457CDA00F086F882F84711DE
:10825000F8E700F08CF8FFF7DFF90020484570DA06
:1082600000F07AF882F83E11F8E700F080F8FFF7A6
:10827000E6F90020484564DA00F06EF882F83F1114
:10828000F8E700F074F8FFF7FDF90020484558DAE8
:1082900000F062F882F84011F8E700F068F8FFF7A4
:1082A00007FA002048454CDA00F056F882F84111F0
:1082B000F8E700F05CF8FFF70EFA0020484540DAD6
:1082C00000F04AF882F84211F8E700F050F8FFF7A2
:1082D00026FA0020484534DA00F03EF882F84311CF
:1082E000F8E700F044F8FFF737FA0020484528DAAD
:1082F00000F032F882F84411F8E700F033F8FFF7A5
:10830000B9FC002048451CDA00F026F882F8491133
:10831000F8E700F02CF8FFF7C8FC0020484510DA19
:1083200000F01AF882F84811F8E700F020F8FFF79B
:10833000F1FC002003E000F00FF882F84A114845F4
:10834000F9DB284601F086F8204601F083F8029810
:10835000BDE8FE4F01F07EB807FB00F2215C5244FD
:10836000401C70472B465A465146484670472A469D
:108370005146484670472DE9F0470646B046062765
:108380000C4617FB08F091469A460121C0B2F9F756
:1083900071F9050001D13448E2E6504604284FF453
:1083A000A67A04D00E282AD0112839D049E008989E
:1083B000012802D0022811D043E021463046FFF7C1
:1083C000C8FC002040453CDA002100F053F893F847
:1083D000A23000F04BF8F8DB401CF3E721463046B2
:1083E000FFF7F9FC002040452BDA002100F042F8AD
:1083F00093F8B03000F03AF8F8DB401CF3E7214680
:108400003046FFF74DFD002040451ADA002100F00C
:1084100031F893F8203100F029F8F8DB401CF3E73D
:1084200021463046FFF7FFFC002008E0002100F065
:1084300021F893F8BE3000F019F8F8DB401C4045F5
:10844000F4DB3046FEF77EFF2A4649463046FFF70A
:1084500031FE2846BDE8F04700F0FCBFA4BD00088F
:108460007CC6000884C70008D4C50008AB54491C6A
:10847000062970470AFB00F323440B4407FB001254
:1084800070471CB500228DF8002001AC03788DF8F0
:10849000043001A9427862700220FFF729FD010A29
:1084A000A1708DF80700FEF73EFFFEF713FF0421D1
:1084B00001A8FEF717FF01216846FEF72CFF9DF883
:1084C0000000FF28F7D1FEF707FFFEF734FF044650
:1084D000FEF72DFF204616BD5265616420416C6C8D
:1084E00020636D642077726F6E67207479706520E9
:1084F00073656C65637400004661696C6564207423
:108500006F20616C6C6F63617465206D656D6F7257
:108510007900000038B5044600F09EFF14F1010F09
:10852000054602D004480178641800F095FF401B0E
:10853000A042FAD331BD00BF700100202DE9F84FF1
:108540000D4600267449754A0F23044601202F6802
:10855000B04000EA0708804540F0CB804FEA460C67
:10856000032707FA0CF76FEA070E6F68012F18BF91
:10857000022F03D0112F18BF122F12D1A768D5F8E0
:108580000C900EEA070709FA0CF949EA0707A760F9
:10859000676827EA00006F68C7F30017B7403843E1
:1085A0006060E068AF680EEA000007FA0CF7384335
:1085B000E060B0006F68022F18BF122F12D1F708C9
:1085C00004EB870700F01C09D7F820A003FA09FB89
:1085D0002AEA0B0AD5F810B00BFA09F949EA0A0998
:1085E000C7F8209027680EEA070E2F7907F00307D7
:1085F00007FA0CF747EA0E0727606F68FF0078D587
:10860000002700974FEA960C176847F480471760D9
:1086100000F00C00176807F48047009703FA00FE8B
:10862000009F3F4F57F82C7027EA0E0E3D4FBC427B
:1086300008BF00272CD03C4FBC4208BF012727D0E1
:108640003A4FBC4208BF022722D0394FBC4208BF74
:1086500003271DD0374FBC4208BF042718D0364F20
:10866000BC4208BF052713D0344FBC4208BF0627C1
:108670000ED0334FBC4208BF072709D0314FBC4250
:1086800008BF082704D0304FBC420CBF09270A2777
:1086900007FA00F0224F40EA0E0047F82C006FEA7C
:1086A00008000F6800EA070C6F68FF0348BF48EA3C
:1086B0000C0CC1F800C04F6800EA070C6F68BF03DC
:1086C00048BF48EA0C0CC1F804C08F6800EA070CE8
:1086D0006F68FF0248BF48EA0C0CC1F808C0CF68B9
:1086E00000EA070C6868800248BF48EA0C0CC1F831
:1086F0000CC0761C0F2E7FF629AFBDE8F18F02B9B2
:10870000090481617047114A136803421CBF10605D
:1087100000F01EB870470000003C014044380240A1
:1087200008380140000002400004024000080240F6
:10873000000C0240001002400014024000180240E9
:10874000001C02400020024000240240143C014072
:108750007047000038B5040001D1012032BD00206F
:10876000A06204F15005687820B9002129702046E4
:1087700000F044FF0220687000F0E6FA6268A16829
:10878000E06823680A432169024360690A43A169DA
:10879000024301F40071E0690A43216A0243A06ABE
:1087A0000A4302431A60A169606A2268090C01F059
:1087B0000401014351602068C16921F40061C16175
:1087C000002068600121697032BD2DE9F84300F096
:1087D0000DFA984608BF022000F08880012038700A
:1087E00000F03AFE7978012918BF02267CD1002CCE
:1087F00018BFB9F1000F76D0032179707E602C6329
:10880000A5F83490A5F83690AE63AE87EE876E6417
:108810002E64AB68B3F5004F04D129680B6843F4AC
:1088200080430B6029680B685C0603D40B6843F037
:1088300040030B604446E968B1F5006F696821D1D7
:10884000002918BFB9F1010F00F0E5F9804604E0F6
:10885000296B0A88C26000F0BBF9E88E002833D08B
:10886000286881688A07F3D400F0F6FDA0EB0800C1
:10887000A04204D314F1010FEFD0032634E0002C02
:10888000EBD1FAE7002918BFB9F1010F00F0B7F9F1
:10889000804606E0296B0A780273286B411C00F0C1
:1088A00099F9E88E80B1286881688A07F2D400F0CF
:1088B000D3FDA0EB0800A04203D314F1010FF0D0C8
:1088C000DBE7002CEDD1D8E742462146284600F0F0
:1088D000B4FA08B120207860A86810B900F07FF9D8
:1088E000009A786800B1012600F09AF8BDE8F2839A
:1088F0002DE9F843002604460D466068B0F5827FF6
:1089000004BFA06800289146984604F1500709D199
:1089100004267E70CDF800804B462A46204600F0A3
:1089200085F87BE03878012808BF022076D0012046
:10893000387000F091FD7978012918BF02266BD1BB
:10894000002D18BFB9F1000F65D0042179707E6049
:10895000A563A4F83C90A4F83E902663A686E6861C
:1089600026646664A268B2F5004F04D121680A68E3
:1089700022F480420A6021680A68530603D40A6818
:1089800042F040020A600546E168002926D108E06D
:10899000007BA16B0870A06B421CA263E08F411E9C
:1089A000E187E08F68B320688168CA07F0D400F0DF
:1089B00053FD401B404504D318F1010FF1D00326AD
:1089C0002AE0B8F1000FECD1F9E7C068A16B08808C
:1089D000A06B821CA263E08F411EE187E08F80B113
:1089E00020688168CA07F0D400F036FD401B40457E
:1089F00003D318F1010FF1D0E1E7B8F1000FEDD189
:108A0000DDE72A464146204600F0EFF908B1202074
:108A10007860786800B1012600F002F8BDE8F283C2
:108A20000120787000213970304670472DE9FC47ED
:108A300000F0DCF84FF0010808BF022000F0C6800B
:108A40009A4687F8008000F007FD7B78012B09D05B
:108A50006968B1F5827F02BFA9680029042B01D0A3
:108A60000226AEE0002C1CBFB9F1000FBAF1000FD6
:108A700001D10126A5E07B78042B1CBF052179706C
:108A80007E60C5F83890A5F83EA0A5F83CA02C6300
:108A9000A5F836A0A5F834A02E646E6429680C6889
:108AA000630603D40C6844F040040C60E9680A9C37
:108AB000B1F5006F696838D1002918BFBAF1010F0C
:108AC00000F0A9F88146E88E002804BFE88F00284E
:108AD00068D02968886882070BD5E88E002818BFFF
:108AE000B8F1000F05D0286B0288CA60B04600F0CC
:108AF0006FF829688868C2070CD5E88F50B1C8683C
:108B0000A96B08804FF00108A86B821CAA63E88F4C
:108B1000411EE98700F0A0FCA0EB0900A042D2D3DF
:108B200014F1010FCFD003264BE0002918BFBAF192
:108B3000010F00F064F88146E88E002804BFE88F3A
:108B400000282FD02968886882070DD5E88E002874
:108B500018BFB8F1000F07D0286B02780A73B0462F
:108B6000286B411C00F036F829688868C2070CD5CC
:108B7000E88F50B1C868A96B08704FF00108A86B66
:108B8000421CAA63E88F411EE98700F065FCA0EB58
:108B90000900A04203D314F1010FCDD0C3E7002C8C
:108BA000CAD1C0E74A462146284600F046F918B126
:108BB00020200126786004E0A86810B900F00FF8C2
:108BC000009801217970002038703046BDE8F687A2
:108BD000286B811C2963E88E411EE9867047009648
:108BE0002968CA680092896800917047054605F1B6
:108BF00050070026387801280C469146704709D165
:108C0000296B2B680A781A73296B4A1C2A63E98E30
:108C10004A1EEA86704709D1296B2B680A88DA60F8
:108C2000296B8A1C2A63E98E4A1EEA8670477CB546
:108C3000044622685168936803F04100012806D178
:108C4000480604D5216C2046BDE87C4008479807BB
:108C500006D50D0604D5616C2046BDE87C4008476A
:108C600013F4B07F63D0880661D55D060ED594F805
:108C7000510003284ED0606D40F00400606500256F
:108C80000095D66800969568009500989D060DD5CC
:108C9000606D40F0010060650025009592680092CB
:108CA0002068056825F0400505600098DA0509D5BB
:108CB000606D40F0080060650022009220688268C4
:108CC0000092009B606D90B32068426822F0E00241
:108CD0004260012011F0030F84F8510022D0206877
:108CE0000FF24D054168890889004160E06C28B1A8
:108CF0000565E06C00F0F8FD00F020F8A06CB0B164
:108D00000565A06C00F0F0FD88B1606D40F040009A
:108D1000606573BD00200090D16800919268009258
:108D2000009873BD2046BDE8764000F0EFBD73BDEE
:108D3000806B0021C187C18600F0E8BD18B1606D6D
:108D400040F04000606570472068016821F04001F4
:108D5000016070472DE9F041069F05460E4690469A
:108D60001C46286881683140B1420CBF01200020B8
:108D7000404531D014F1010FF3D000F06DFBC01B62
:108D8000A04201D2002CECD12868416821F0E0011A
:108D900041606868B0F5827F08D1A868B0F5004FDF
:108DA00018BFB0F5806F01D100F019F8A86AB0F5CE
:108DB000005F09D12868016821F40051016028682A
:108DC000026842F40052026005F150000121417036
:108DD00000220270032000E00020BDE8F081286836
:108DE000016821F04001016070471CB504460B4644
:108DF0006068B0F5827F08D1A068B0F5004F18BF59
:108E0000B0F5806F05D1FFF79FFF6068B0F5827FF6
:108E100007D1A0680092B0F5806F03D000228021B6
:108E200002E00092002201212046FFF793FF10B1DB
:108E300000F02BF816BD002016BD7CB50446164880
:108E4000164E0B4601681825B1FBF5F5B5FBF6F695
:108E50004FF47A70464300966168B1F5827F09D17C
:108E60000092802100222046FFF774FF58B100F0E5
:108E70000CF876BD009830B10098401E0090216833
:108E800088680106F6D4002076BD606D40F02000B1
:108E900060650320704700007C01002040420F0005
:108EA00038B5040001D1012032BD00F058F818B9DE
:108EB00000F051F800F01EFC36E0022180F83D1071
:108EC0000268916801F00701062904D001680A6868
:108ED00042F001020A6012E0022180F83D1041F2E6
:108EE000111301680A6A1A4202BF096A40F2444239
:108EF000114204D101680A68520852000A60012137
:108F000080F83D10002070470068C16841F0010101
:108F1000C160816801F00701062903D0016841F0B2
:108F2000010101600020704702206870211D206847
:108F300000F0AEF901206870002032BD38B50400A1
:108F400001D1012032BD00F00AF818B900F003F891
:108F500000F0DDFCE8E7002129702046704704F1AD
:108F60003C056878704710B50446206801698A0797
:108F700015D5C1688A0712D56FF00201016101227F
:108F80002277806910F0030F204602D000F0C0FC69
:108F900003E000F0BEFC00F087F800202077206896
:108FA00001694A0715D5C1684A0712D56FF0040157
:108FB000016102222277806910F4407F204602D0AE
:108FC00000F0A6FC03E000F0A4FC00F06DF8002027
:108FD0002077206801690A0715D5C1680A0712D5EC
:108FE0006FF00801016104222277C06910F0030FBD
:108FF000204602D000F08CFC03E000F08AFC00F078
:1090000053F80020207720680169CA0615D5C16889
:10901000CA0612D56FF01001016108222277C069DB
:1090200010F4407F204602D000F072FC03E000F014
:1090300070FC00F039F80020207720680169CA0729
:1090400008D5C168CA0705D56FF001010161204646
:1090500000F015FF206801690A0608D5C1680A06F4
:1090600005D56FF080010161204600F03FFF2068C8
:1090700001694A0608D5C1684A0605D56FF0400166
:109080000161204600F033FF206801698A060AD595
:10909000C1688A0607D56FF0200101612046BDE84E
:1090A000104000F025BF10BD204600F022BFF8B5EB
:1090B00000F07FF801D10220F2BD00F087F882B9FC
:1090C000EB686A682968306800F02DF930688169BA
:1090D00021F00C01816131688A69A86802438A61C4
:1090E0005CE0042A10D1EB686A682968306800F0F7
:1090F00072F93068816921F4406100F056F8AA687D
:1091000041EA0221816149E0082AE9686A682B681E
:1091100023D13768386A20F4807038621B0207F167
:109120001C0003F42063D0F800C0D7F820E04FEA19
:109130009C0C42EA8C0261F3071202602EF420605C
:1091400003433B623068C16921F00C01C1613168A1
:10915000CA69A8680243CA6120E030681C301B035A
:10916000476827F48057476003F420430768D0F826
:1091700004C027F4407747EA022761F30F372CF445
:10918000204107600B4343603068C16921F44061AE
:1091900000F007F8AA6841EA0221C16100F010F866
:1091A000F2BDC1613068C169704781613068816911
:1091B0007047064606F13C040D46207801287047AA
:1091C0000120607000212170002070470120207074
:1091D00002216170704738B500F04EF801D10220CD
:1091E00032BD0120207002226270DFF89C012A68E3
:1091F0009368034093600868020018BF10282DD0C0
:10920000202818BF302829D0402823D0502816D035
:10921000602818D0702803D0B0F5005F07D021E097
:1092200000F025F82868816841F0770105E000F03A
:109230001EF82868816841F48041816012E000F0E6
:1092400012F850210BE0CA684968286800F0D9F884
:10925000602104E000F007F8402100E001462868A2
:1092600000F0E1F80EE0CA6849682868A4E0CB681D
:109270004A6889682868DEE0054605F13C042078E4
:10928000012870470120607000212170002032BD4C
:10929000F0B53E4C05683E4B3E4E3F4FDFF8FCC0FC
:1092A000A04218BFB0F1804F07D0604518BFB84248
:1092B00003D0B04218BF98420DD14A6825F070051E
:1092C0001543A04218BFB0F1804F17D060451CBFB6
:1092D000B842B04212D098421CBF314A90420DD0E1
:1092E000304EB0421CBF304A904207D02F4EB042A1
:1092F0001FBF2F4A90422F4EB04203D1CA6825F4B7
:10930000407515434A6925F0800515430560A04264
:109310008D68C5620A68826212BF9842096901635A
:1093200001224261F0BDF0B5046A184E6408640081
:109330000462B0428469056A18BFB0F1804F11D051
:10934000164EB0421CBF144FB8420BD0114EB04263
:109350001CBF0F4FB84205D0114EB0421CBF134F77
:10936000B84203D1A40842EA840201E044F00102B9
:1093700063F3071225F00A0501F00A01826129430F
:109380000162F0BD000000008800FFFF0000014006
:1093900000040140000C00400008004000040040B0
:1093A00000400140004401400048014000180040D6
:1093B000001C00400020004010B5036A046A6408E5
:1093C0006400046223F00A03846924F0F00444EA90
:1093D0000214846139E030B5046A24F01004046298
:1093E00009018469056A24F4407444EA022463F3A1
:1093F0000F3425F0A00501F0A0018461294301622A
:1094000030BD10B5036A23F0100303628369046A58
:1094100023F4704343EA023324F0A004836144EA56
:109420000114046210BD826822F07002114341F001
:1094300007018160704710B5846824F47F4421439C
:10944000114341EA0321816010BD1943016210BD3F
:1094500000F050BDF7F776BE01484068704700BF86
:109460007001002080B5002000900022DFF8380451
:10947000416841F480414160416801F4804100F05D
:109480004AF80021036843F080530360006800F04D
:10949000805000900098012000F04EFDBDE8024091
:1094A000012000F066BD10B586B000F06EF92168AD
:1094B000DFF8F80381422CD10022DFF8F403009298
:1094C000416941F480714161416901F4807100F0AA
:1094D00022F800F0CBF900F01EF83221036843F0C7
:1094E00001030360032200F04AF9DFF8C803019189
:1094F00002920021039101A9FFF720F854200321D3
:10950000019002910022039201A9DFF8AC03FFF75A
:1095100015F806B010BD009100990092704710B583
:1095200086B000F0D6F82068DFF89013DFF88043AB
:1095300088421BD1002005901222216841F00201CF
:1095400021604FF4C071206800F00200059005987A
:10955000DFF86C0300F047F800200590216941F422
:1095600000112161206900F4001038E0DFF8541385
:10957000884236D100200590216841F00401216025
:109580000021206800F004000590059805914FF433
:109590000071226842F0800222601222206800F0EE
:1095A000800005900598DFF80C0300F01CF81221EC
:1095B0000191012202928020032100900391042254
:1095C00004926946DFF80003FEF7B8FF002005901B
:1095D000216941F400012161206900F40000059037
:1095E000059806B010BD009101920121029103225D
:1095F0000421049103926946FEF7A0BF10B586B01E
:1096000000F067F82168DFF8C422DFF8A402914275
:109610002DD100210591426942F48052426100221D
:10962000416901F4805100F01DF9036843F0020321
:109630000360016801F0020100F014F9182100F044
:109640001DF99F4800F04BF802210191002202927F
:10965000802000F037F89848FEF770FF00220021C4
:10966000232000F069FC232000F083FC28E0984AC6
:10967000914225D100210591426942F48012426154
:109680000022416900F0ECF8036843F02003036016
:10969000016801F0200100F0E5F84FF4407100F09E
:1096A0007AF8059005988B4800F019F8022101918D
:1096B00000220292402000F005F88348FEF73EFFAA
:1096C00006B010BD03210090039105220492694663
:1096D00070470446142200216846FCF79ABD0091A9
:1096E000019200210291032205210491039269460F
:1096F000FEF724BF10B586B000F047F821686C482B
:10970000B1F1804F17D100210091026942F00102AE
:1097100000F0A2F801F00101FFF7FDFE202103682F
:1097200043F001030360022200F029F8624800F0D0
:1097300020F8012117E0684A914218D100210091D8
:10974000026942F0080200F087F801F00801FFF713
:10975000E2FE4FF4806100F01EF8009000985A4835
:1097600000F007F80221059101A9FEF7E7FE06B017
:1097700010BD01910292002103910491704700688D
:1097800000F0010000900098704704461422002168
:1097900001A8FCF73EBD036843F08003036002228A
:1097A000006800F08000704710B586B0FFF791FFA9
:1097B00021684A4A3E48914217D100210591026929
:1097C00042F4002200F048F801F4002100F04AF8C9
:1097D000032100F053F8384800F05BF80022002124
:1097E000342000F0A9FB342032E03D4A914231D1CF
:1097F00000210591026942F4801200F02DF800F07A
:109800002FF800F033F800F02DF84FF48051036882
:1098100043F0080303600222006800F0080005908E
:109820000598244800F035F80221019101220292A6
:1098300004200321009003910822049269462948DC
:10984000FEF77CFE00220021352000F075FB35205C
:1098500000F08FFB06B010BD026100220169704765
:1098600001F480110591059905927047036843F052
:1098700004030360016801F004017047036843F0CA
:10988000010303600222006800F0010005900598C2
:109890007047009101920121029103220821049155
:1098A00003926946FEF74ABE40380240002001405C
:1098B00030380240000802400000024000540040DE
:1098C00000040240005C0040001C024000300140E7
:1098D0000050014000140240000C0040004C0040C9
:1098E00000500040000C024090F83510022903D0CF
:1098F0008022426501207047052180F835100068FC
:10990000026852085200026000207047704770479A
:10991000704770472DE9F84F8AB000F03FFB00F028
:1099200063FA1421684600F053FB0020059048F2CA
:10993000400BDFF85805DFF858450168DFF854554B
:10994000DFF85465DFF85475DFF85485DFF8549577
:10995000DFF854A541F002010160026802F0020242
:109960000592002205990592036843F00403036001
:10997000016801F0040100F032FA43F001030360D2
:10998000016801F0010100F02AFA43F0400303608E
:10999000016801F0400100F022FA43F40073036013
:1099A000016801F4007100F01AFA43F48063036067
:1099B000016801F4806100F012FA43F008030360CB
:1099C000016801F0080100F00AFA43F02003036087
:1099D000016801F0200105910599059201220368B3
:1099E00043F0800303604FF40041006800F0800002
:1099F000059005982046FEF782FE01225946DFF8C1
:109A0000AC04FEF77CFE00224FF460612846FEF7AE
:109A100076FE0022F0213046FEF771FE00224FF460
:109A200040612046FEF76BFE012208213046FEF71A
:109A300066FE0122C0213846FEF761FE0122402168
:109A40004046FEF75CFE00224FF480514846FEF788
:109A500056FE00222B215046FEF751FE01220192B4
:109A600002924FF4004100F0ADF92046FEF766FD8A
:109A700001200321019002900391CDF800B06946C6
:109A8000DFF82804FEF75AFD4FF4606100F09FF9FB
:109A90002846FEF753FD4FF4E0400021009001916D
:109AA000029150466946FEF749FD4FF4805000216F
:109AB00000900191029120466946FEF73FFDF82192
:109AC00000F085F93046FEF739FD4FF4406100F0B3
:109AD0007EF92046FEF732FD012201920292C0215A
:109AE00000F070F93846FEF729FD8020F04900F0BB
:109AF00063F92846FEF722FD0122019202924021DD
:109B000000F060F94046FEF719FD1020032100F037
:109B100053F95046FEF712FD4FF4805100F057F90B
:109B20004846FEF70BFD202100F051F95046FEF7A4
:109B300005FD0B21009101220192022102910022D8
:109B4000039269465046FEF7F9FC002200211720D7
:109B500000F0F2F9172000F00CFAD64CD64804F1C8
:109B600030054FF48271A861E961002028626862C3
:109B7000A862E86220214FF4007028636963002026
:109B8000A863E86328640A21696404F14800FEF7C9
:109B9000E1FD04F1B006C948C949B064F164002090
:109BA00030657065F06530667066B0664FF480476A
:109BB000B76504F1F80000F00FFA04F5A678C14883
:109BC000C8F854000C210020C8F85C00C8F86000F8
:109BD000C8F86400C8F86C00C8F870004FF4E13AA7
:109BE000C8F86810C8F858A004F5D07000F09CFAC6
:109BF00004F5F079B448C9F8000000210C20C9F838
:109C00001400C9F80810C9F80C10C9F81010C9F8E8
:109C10001810C9F81C10C9F804A0484600F084FACE
:109C200006A80021002200238C4680E80E1002A81E
:109C300080E80E10CDE9001204F5187AA349CAF89D
:109C40000010CAF80420CAF808204FF0FF3BCAF8F9
:109C50001020CAF81820CAF80CB05046FFF720F9B7
:109C60004FF48050069006A95046FFF7B4FA5046CC
:109C7000FFF764F90021009101915046694600F018
:109C800013FC01220392002102910491002205920B
:109C900002A95046FFF70BFA8D4828674FF48271EE
:109CA0000020A867E867306069672020F060002224
:109CB0000A204FF40071F0617260B160326172612C
:109CC000B26104F1A000FEF745FD82487C49C8F866
:109CD00000000022C8F80410C8F80820C8F80C20BA
:109CE000C8F81420C8F81820C8F81C20C8F820208C
:109CF000C8F81070404600F06FF968460021002255
:109D00000023002680E84E00734921606260A26053
:109D10002261227684F82020E262E2602A702046E6
:109D20006E49A16200250121E161616100F002FC40
:109D3000022001210090019102966946204600F020
:109D4000ADFC06A800210022002380E82E0002A816
:109D500080E82E00CDE90012C9F844204FF0804180
:109D6000C9F84010C9F84820C9F85020C9F858204F
:109D700004F50874C9F84CB02046FFF791F84FF489
:109D80008050069006A92046FFF725FA2046FFF7E7
:109D9000D5F8009501956946204600F085FB012223
:109DA0000392029500220592049502A92046FFF72E
:109DB0007EF900F023FDFEE700900191002202925F
:109DC00069467047009103220392694670470091EB
:109DD0000122002102910391019269467047059189
:109DE000059905920368704700B593B0342106A821
:109DF00000F0EEF8142101A800F0EAF8002000902D
:109E000001233748016841F080510160002100685A
:109E100000F080500090009832480091026822F4CF
:109E2000404242F4004202600222006800F44040D6
:109E3000009006A80099069210210A910C92002128
:109E40000D91082280210E920F9102220421099384
:109E500010921191129200F04BFE02210291002209
:109E600003920F204FF4A051019004914FF48052BF
:109E70000592042101A800F0A7FF13B000BD0068FF
:109E80001949884208BF01F091B870473038024044
:109E90000000024000180240002802400008024072
:109EA00000140240000C0240002402400004024062
:109EB0000000211040030020003001400054004009
:109EC000A0860100004C004000500040000C004003
:109ED00000500140005C0040002001400100000FE4
:109EE0004038024000700040000001407047704759
:109EF00070477047074601F061F83846F7F728FCCD
:109F0000FBE700000901020002D41F48815470479A
:109F10001E4B02F00F021A4402F8041C70471C4B3F
:109F200019684FF6FF020002114000F4E060084398
:109F3000184908431860704770B5154B1C68C4F386
:109F400002230124C3F10705052D2EBF0F2504FAB6
:109F500005F56D1E1E1D072E34BF0023DB1E294094
:109F6000994004FA03F3BDE870405B1E1A401143A8
:109F7000C8E7010007D4012200F01F01064B8A4008
:109F8000400943F82020704700E400E018ED00E0AD
:109F90000CED00E00000FA0500E100E080B50B48A0
:109FA000016841F400710160026842F4806202605D
:109FB000016841F4807101600320FFF7B0FF0020C9
:109FC00001F01AF8FFF74EFA002002BD003C0240F3
:109FD000002201F04FB80000F8B5040025D004F1CC
:109FE0003C05697821B9002028702046FFF797FAD0
:109FF00024216970206802685208520002602068BB
:10A00000016841F4004101602068026822F40042C6
:10A01000026000F05FFF01466068DFF8F4209042C4
:10A0200005D2DFF8F030994205D20120F2BDDFF809
:10A03000E8008142F9D32068DFF8E0304668B1FBE0
:10A04000F3F3B60943EA861646602668376A606805
:10A05000904206D34FF4967043434FF47A70B3FBAB
:10A06000F0F35B1CBF0943EA87133362491E236880
:10A07000DE696768974206D27F0000F043F8042942
:10A0800013D2042111E0A06820B907EB470700F0C4
:10A0900039F805E01920474300F034F841F48041D5
:10A0A00008050CBF012141F40041DFF874000640AF
:10A0B0000E43DE6122681368E169206A23F0C00361
:10A0C0000B43034313602268DFF85800936821694B
:10A0D0000340E0680B43034393602168CA68A369A7
:10A0E0006069120A034343EA0222CA6020680168D9
:10A0F00041F0010101600020686020216970206347
:10A10000A870F2BDB1FBF7F1491CC1F30B01704718
:10A11000A186010080841E0000093D0040420F001E
:10A120000030FFFF007CFFFF38B5040001D10120A3
:10A1300032BD00F021F808B900F022F800F012F862
:10A1400000F023F8FFE7416100F001F832BD20681C
:10A15000C16841F40051C16000206860202169702D
:10A16000A9707047242068702068C16821F40051EC
:10A17000C160204600F025B904F1380568787047C1
:10A18000002129702046FFF70FBB2068016921F4E8
:10A19000904101612068416921F02A0170474169BD
:10A1A00021F040014161606B704770B50446206842
:10A1B0000368C668456913F00F0206F0200003F03B
:10A1C000200107D1002918BF00285BD02046BDE838
:10A1D0007040ADE0EA0702D416F4907F52D0DA075F
:10A1E00005D5F60503D5E26B42F00102E2635A079A
:10A1F00005D5EE0703D5E26B42F00202E2639A074F
:10A2000005D5EE0703D5E26B42F00402E2631A07BC
:10A2100006D508B9EA0703D5E36B43F00803E36307
:10A22000E26B002A6ED000291EBF0028204600F0F5
:10A230007FF820684069E16B0A0701D440061BD50E
:10A24000204600F060F8206841694A060FD5FFF704
:10A25000A6FF60B10FF2CD010165606BFFF744FB13
:10A2600000284FD0606B016DBDE870400847204664
:10A27000BDE8704000F017BF204600F014FF00203A
:10A28000E06370BD18062CD531062AD594F8390044
:10A29000212837D1A068B0F5805F206A0CD10188F1
:10A2A0002268C1F30801516020690028206A0CBFB0
:10A2B000811C411C216204E0411C2162226800785B
:10A2C0005060E08C401EE08480B2D8B92068C1683C
:10A2D00021F08001C1602068C16841F04001C16087
:10A2E00070BD58060ED571060CD52068C16821F0E6
:10A2F0004001C1602046202184F83910BDE870403B
:10A3000000F0D2BE70BD0168CA6822F49072CA60C3
:10A3100001684A69520852004A61202180F83A10C7
:10A3200070470000806B0021C185C18400F0BBBE76
:10A3300010B590F83A10222941D18168B1F5805FBB
:10A340002AD1826A0169134601BB04686168C1F3BE
:10A350000801921C82621980C18D491EC18589B293
:10A3600059BB0168CA6822F02002CA600168CA6845
:10A3700022F48072CA6001684A69520852004A6138
:10A38000202180F83A1000F090FE16E0016849683C
:10A3900001F0FF01521CDDE701690029816A05D146
:10A3A0004A1C826203685A680A70D5E74A1C8262B6
:10A3B00003685A6802F07F02F6E7002010BD022011
:10A3C00010BDD0B50646642732681169F06821F4E3
:10A3D0004051014311611924D3682D48B1680340ED
:10A3E00030690B4371690343F0690B430343D36046
:10A3F0005169B06921F4407101435161F369254805
:10A400002549B3F5004F1FD18A4218BF824202D1BD
:10A4100000F068FD01E000F05DFD0246A4FB0201D2
:10A420007268D30F5200FBF797FA00F037F8FF007D
:10A4300032376420B7FBF0F0420002F4F87202EB0E
:10A44000011200F007001DE08A4218BF824202D1CB
:10A4500000F048FD01E000F03DFD0246A4FB0201D2
:10A460007268930F9200FBF777FA00F017F83F013C
:10A4700032376420B7FBF0F000F0F00202EB01127B
:10A4800000F00F00316880188860D0BD0000000027
:10A49000F369FFFF00140140001001406421B0FB8C
:10A4A000F1F107FB1107704770B500F13C031A7812
:10A4B000012A01D1022070BD01221A7002245C70B1
:10A4C00005686E68AC680A6826F0700616436E6010
:10A4D00002681148824218BFB2F1804F11D00F4874
:10A4E00082421CBF0E4DAA420BD00E4882421CBFB6
:10A4F0000D4DAA4205D00D4882421CBF0C4DAA4208
:10A5000004D1486824F08004044394600121597008
:10A510000020187070BD00000000014000040040E1
:10A5200000080040000C00400004014000400140D1
:10A530000018004070B5044600250CB9012070BD1C
:10A5400004F13006306920B92046FEF7ACFF756192
:10A5500035733069C10600F192803069DFF88412EA
:10A5600020F4885040F002003061086820F4403048
:10A5700008600A68606802430A602068416821F444
:10A580008071416020684168226941EA022141608E
:10A590002068416821F04071416021684A68A068E4
:10A5A00002434A602068816821F40061816021686B
:10A5B0008A68E06802438A602068A16ADFF828227E
:10A5C0009142816821F0706181600CD021688A68B5
:10A5D000A06A02438A6000F05BF821688A68E06A3A
:10A5E00002438A6001E000F053F82068816821F09E
:10A5F000020100F049F8227E41EA4201816094F8AC
:10A6000020002168002848680FD040F400604860AE
:10A610002068416821F46041416020684168626AB5
:10A62000521E41EA4231416002E020F4006048607D
:10A630002068C16A21F47001C1622068C16AE269C0
:10A64000521E41EA0251C1622068816821F4007102
:10A6500000F01AF8327841EA422100F015F821F4AE
:10A66000806100F011F8626941EA822181607561C0
:10A67000316921F0020141F00101316100E0012561
:10A6800000203073284670BD816020688168704763
:10A690002068816821F040518160704778B502469A
:10A6A0000020009092F83C30012B01D1022072BDB5
:10A6B000012082F83C0007240B6810680A2B12D393
:10A6C0000A3BC56803EB43039C4025EA0404C460CD
:10A6D000C3680D688C68A5F10A0606EB4606B4400F
:10A6E0002343C3600FE0056903EB430304FA03F35C
:10A6F00025EA0303036103690D688C6805EB4505D2
:10A70000AC40234303611F244B68072B0CD25B1E14
:10A71000456B00F059F84463436B4D680C886E1E1E
:10A7200000F04DF843631BE00D2B0CD2DB1F056BD3
:10A7300000F04AF80463036B4D680C88EE1F00F0CC
:10A740003EF803630CE00D3BC56A00F03DF8C462BF
:10A75000C36A4D680C88A5F10D0600F030F8C3629D
:10A76000224B984226D10C681E48122C07D1036850
:10A7700023F400030360046844F4800404600B685D
:10A780001D4CA34218BF112B14D1036823F480037E
:10A790000360056845F4000505600868A04209D11A
:10A7A0001449134C0B68B3FBF4F40A20444300949F
:10A7B00000F010F8002182F83C10002072BD06EB7A
:10A7C0008606B4402343704703EB83039C4025EA8D
:10A7D0000404704702E00098401E00900098002892
:10A7E000F9D17047042301400100000F002001400F
:10A7F00040420F007C010020120000101CB5F7F74A
:10A80000C2FFAB4C6846F8F753F800F05BF9FBF772
:10A8100085FF009800F002F8F4E7000010B501464B
:10A820002329A448A24C00F23D81DFE811F0370152
:10A8300024002B00320037003C00410046004B0052
:10A84000500057006B00720086008D00A100A80028
:10A85000BE00C300CA00D100D800DF00E400EB0056
:10A86000F200F900000105010A010F0114011B01AA
:10A8700022012901300104F10C01BDE81040012042
:10A88000FBF756BF04F10C01BDE810400120FBF7B7
:10A8900081BFBDE810400120FBF794BFBDE8104028
:10A8A0000120FBF7B6BFBDE810400120FBF79CBFBD
:10A8B000BDE810400120FBF7C3BFBDE810400120F8
:10A8C000FBF7D5BFBDE810400120FBF7E9BF04F15D
:10A8D0000C01BDE810400120FBF7F7BF00F0F6F8CF
:10A8E00000F0EDF8A0682168884251DAF7F7DBFF45
:10A8F00000F0E8F8FBF7E9FF00F0DEF8A068401C84
:10A90000A060EFE704F10C01BDE810400120FBF767
:10A91000F9BF00F0DBF800F0D2F8A06821688842A7
:10A9200036DAF7F7C0FF00F0CDF8FBF7EBFF00F0E9
:10A93000C3F8A068401CA060EFE704F10C01BDE87B
:10A9400010400120FBF7F5BF00F0C0F800F0B7F8A9
:10A95000A068216888421BDAF7F7A5FF00F0B2F87B
:10A96000FBF7E7FF00F0A8F8A068401CA060EFE745
:10A9700004F10C01BDE810400120FBF7FABFF7F726
:10A980007AFF00F09CF80020A0602168A06888424F
:10A9900080F28D80F7F787FF00F094F8FBF7E9FF6E
:10A9A00000F08AF8A068401CEEE7BDE810400120E6
:10A9B000FCF74EB804F10C01BDE810400120FCF793
:10A9C00056B804F10C01BDE810400120FCF769B84D
:10A9D00004F10C01BDE810400120FCF76EB804F151
:10A9E0000C01BDE810400120FCF7BFB8BDE81040E5
:10A9F0000120FCF7D2B804F10C01BDE810400120A1
:10AA0000FCF7D9B804F10C01BDE810400120FCF7B7
:10AA1000E0B804F10C01BDE810400120FCF7E9B8F2
:10AA200004F10C01BDE810400120FCF712B9BDE8AB
:10AA300010400120FCF71EB9BDE810400120FCF7D2
:10AA400026B9BDE810400120FCF72EB9BDE8104042
:10AA50000120FCF736B904F10C01BDE810400120DB
:10AA6000FCF73CB904F10C01BDE810400120FCF7F3
:10AA7000CFB904F10C01BDE810400120FCF7E4B9A6
:10AA800004F10C01BDE810400120FCF743BA04F1C9
:10AA90000C01BDE810400120FCF785BABDE810406C
:10AAA000F7F771BEBDE810400AA0F7F7E4BE10BD8D
:10AAB00010000020A8C700086068FCF709BC204609
:10AAC000F7F7F6BE04F10C01012070470021A160E8
:10AAD000F7F7D1BE496E636F7272656374204F7071
:10AAE00074696F6E0000000000200860FEF7B4BCBF
:10AAF0002DE9F8430646DFF8C0523078C1074AD541
:10AB0000A86800F00C00042807D0A86800F00C002A
:10AB100008280AD16868410207D5286881033AD518
:10AB20007068002837D101203CE17068B0F5803FA3
:10AB300004D1286840F48030286011E0B0F5A02FDF
:10AB4000286806D140F480202860296841F48031CB
:10AB500005E020F480302860296821F480212960F4
:10AB6000706860B1FEF778FC04462868810312D44F
:10AB7000FEF772FC001B6528F7D3032012E1FEF7F5
:10AB80006BFC04462868810305D5FEF765FC001BB5
:10AB90006528F7D3F1E73078894F810718D5A86881
:10ABA00010F00C0F07D0A86800F00C00082823D183
:10ABB0006868410220D42868810702D5F06801281E
:10ABC000B1D12968306921F0F80141EAC00129605A
:10ABD0003178080741D570697A4990B301220A603B
:10ABE000FEF73AFC0446686F810736D4FEF734FC62
:10ABF000001B0228F7D9C0E7F068A8B1012139602D
:10AC0000FEF72AFC04462868810705D4FEF724FCD9
:10AC1000001B0228F7D9B0E72868316920F0F80056
:10AC200040EAC1002860D3E73860FEF715FC04460F
:10AC300029688807CCD5FEF70FFC001B0228F7D93E
:10AC40009BE7FFF752FF0446686F810705D5FEF7C3
:10AC500003FC001B0228F7D98FE7307841075ED547
:10AC6000286C0024C1000AD400940124296C41F00E
:10AC700080512964286C00F0805000900098DFF823
:10AC80003C81D8F80000C10512D4D8F8000040F487
:10AC90008070C8F80000FEF7DFFB8146D8F800009E
:10ACA000C10505D4FEF7D8FB00F082F8F6D964E7B9
:10ACB000B068012805D00528286F06D140F00400AF
:10ACC0002867286F40F0010005E040084000286731
:10ACD000286F20F00400286741F28938B06860B11D
:10ACE000FEF7BAFB8146286F810713D4FEF7B4FB49
:10ACF000A0EB09004045F6D33FE7FEF7ADFB8146E8
:10AD0000286F810706D5FEF7A7FBA0EB0900404599
:10AD1000F6D332E71CB1286C20F080502864B0696B
:10AD200000283ED0A96801F00C0108293FF4FBAED1
:10AD300002282AD100F038F804462868810105D598
:10AD4000FEF78AFB001B0228F7D916E7F069316A83
:10AD5000726A0843B16A490840EA8210491E40EA13
:10AD60000140F16A326B40EA016040EA02706860BB
:10AD7000012000F01AF804462868810111D4FEF77A
:10AD80006BFB001B0228F7D9F7E600F00DF804462C
:10AD90002868810105D5FEF75FFB001B0228F7D963
:10ADA000EBE60020BDE8F28300203866FEF754BBD6
:10ADB000A0EB0900022870470038024000700040F4
:10ADC00000004742800E47422DE9F04104000F4643
:10ADD00054D0574E306800F00F00B84202D200F055
:10ADE00073F84BD12068534D810712D5400703D526
:10ADF000A96841F4E051A9602078010703D5A8684B
:10AE000040F46040A860A968A06821F0F001014307
:10AE1000A9602178C80729D56068012802D129686E
:10AE20008A0305E0022818BF032803D129688A0194
:10AE300003D423E029688A0720D5A968890840EA55
:10AE40008100A860FEF708FB8046A868616800F0F2
:10AE50000C00B0EB810F09D0FEF7FEFAA0EB080062
:10AE600041F289318842F0D303202BE0306800F0B2
:10AE70000F00874204D200F027F801D0012021E022
:10AE80002078410705D5AA68E06822F4E052024321
:10AE9000AA602178080706D5A968206921F46041D5
:10AEA00041EAC001A96000F051F8AA682249234B89
:10AEB000C2F30312895CC84018602148006800F0A2
:10AEC0009BF80020BDE8F0813770316801F00F0178
:10AED000B942704719481B4A006813681A49C3F3FE
:10AEE000822206E01548174A006813681649C3F322
:10AEF0004232895CC840704710B50F220260114A87
:10AF0000136803F003034360146804F0F0048460E2
:10AF1000136803F4E053C3601268D20802F4E052ED
:10AF200002610348026802F00F020A6010BD0000CF
:10AF3000003C02400038024014C500087C0100209B
:10AF40007801002008380240A4C8000830B5144C2D
:10AF5000606800F00C00042802D0082802D01DE030
:10AF6000104830BD226820680023410202F03F02F1
:10AF700004D525680B49C5F3881003E020680A4909
:10AF8000C0F38810A1FB0001FAF7E6FC2168C1F3C9
:10AF90000141491C4900B0FBF1F030BD024830BD11
:10AFA0000438024040787D010024F40002484168E2
:10AFB00002788A18426070477001002038B50D4D44
:10AFC0000824286800281CBF017811F0030F05D061
:10AFD00090F90310002958BF00F068F82D1D641E79
:10AFE000EFD1BDE83840002200214FF0FF3000F0E3
:10AFF0009CB800BFD802002018B5014687B00022D7
:10B000001920FEF799FF1920FEF7B3FF00200090EA
:10B01000144C1548016841F00101016001A9006864
:10B0200000F001000090009802A8FFF765FFFFF70D
:10B0300059FF0E49216040F2E73240000C49E260BE
:10B04000B0FBF1F0401E606000222261A260204649
:10B05000FDF726FF18B92046FDF756FF00E0012056
:10B0600008B010BDD808002044380240000001405C
:10B0700040420F0000B500BF1300964694461039B9
:10B0800028BFA0E80C50FAD85FEA417C28BF0CC06A
:10B0900048BF40F8042BC90728BF20F8022B48BF3F
:10B0A00000F8012B00BD70477047704738B50400A9
:10B0B0000ED0207810F0030F03D094F9030000287D
:10B0C00009D5AFF30080204600F038F8AFF30080D8
:10B0D0004FF0FF3032BD204600F0B8F80546AFF320
:10B0E00000802078410644BF6068FEF7B3F9002075
:10B0F000606094F90300022804D900F0C3F808B195
:10B100004FF0FF35E06B48B100F0C8F808B14FF0E0
:10B11000FF35E06BFEF79EF90020E063204600F06B
:10B120000DF8AFF30080284632BD80B5002802D468
:10B1300000F0BEF802BD002002BD000082B0017820
:10B140000A062FD523490B6800930022834203D1BE
:10B15000002341F8223022E04B6800930122834211
:10B160001FBF02228B6800938342F1D0CB6800930B
:10B17000032283421FBF04220B6900938342E7D05E
:10B180004B690093052283421FBF06228B690093FF
:10B190008342DDD00722CB6900938342D8D002B02E
:10B1A000FEF758B9002101804FF0FF3200F1440151
:10B1B000C270C1604161C16100F1440300F1440209
:10B1C00000F130014360026182610262416202B0BB
:10B1D00070470000D802002070B50546AFF300802C
:10B1E000288881042DD56E68002400E00644EA68B2
:10B1F00095F903003146914208D2521AFFF795FFA4
:10B2000010F1010F09D00028F0D106E00022002142
:10B21000FFF78BFF10F1010F00D101246868E8608F
:10B22000A861E861298844B141F400712980284669
:10B23000AFF300804FF0FF3070BD4DF6FF7001405E
:10B2400029802846AFF30080002070BDF8B5A0B972
:10B25000AFF3008000250A4E08244FF0FF37306816
:10B2600020B1FFF7B9FF002848BF3D46361D641ED8
:10B27000F5D1AFF300802846F2BDBDE8F240ABE760
:10B28000D80200201CB50200009269460220ABBE25
:10B290000400100000F01CF8200016BDE0B500907E
:10B2A000FAF7C8F9019069460E20ABBE03B000BDA5
:10B2B00080B5002901D1002002BD012801D002285B
:10B2C00002D100F06BF802BD00F078F802BD00007A
:10B2D00010B4314A002113461C6884421EBF491C29
:10B2E0009C6884421EBF491C1C69844209D09C6929
:10B2F000491C844205D0491C20331029ECD310BCD2
:10B300007047002342F8313002EBC1014B6010BCA2
:10B31000704770B4204C002325462E688E421EBF15
:10B320005B1CAE688E421EBF5B1C2E698E4209D02C
:10B33000AE695B1C8E4205D05B1C2035102BECD314
:10B3400070BC7047054604EBC303012A04BF59686B
:10B350004D195D6070BC704710B40F4A0021134650
:10B360001C6884421EBF491C9C6884421EBF491C45
:10B370001C6984420AD09C69491C844206D0491C3D
:10B3800020331029ECD310BC0020704702EBC10021
:10B39000406810BC70470000B807002030B583B08B
:10B3A0000C0015000120F6F727FA00900194029591
:10B3B00069460520ABBE281A03B030BD18B583B06E
:10B3C0000300140000930191029469460520ABBE6E
:10B3D00001221900201AFFF79CFF04B010BD0000E5
:10B3E000577269746520616E642052656164204300
:10B3F0006F6E66696775726174696F6E3A2031208D
:10B40000202020202020202020202020202020203C
:10B41000202020202020202020202020207C526559
:10B42000616420446576696365205349443A20325B
:10B4300036202020202020202020202020202020F6
:10B4400020200A005265616420436F6E666967754B
:10B45000726174696F6E3A203220202020202020F3
:10B4600020202020202020202020202020202020DC
:10B4700020202020202020202020202020202020CC
:10B48000207C536F66742052657365743A2032379E
:10B4900020202020202020202020202020202020AC
:10B4A0002020202020200A0053746172742041441F
:10B4B000493120436F6E76657273696F6E285369E8
:10B4C0006E676C652053686F74293A203320202002
:10B4D000202020202020202020202020202020206C
:10B4E00020202020207C526573657420636D6420C9
:10B4F000636F756E7465723A2032382020202020E8
:10B50000202020202020202020200A005374617257
:10B5100074204144493220436F6E76657273696FBF
:10B520006E2853696E676C652053686F74293A20E2
:10B5300034202020202020202020202020202020F7
:10B540002020202020202020207C534E41502853B2
:10B55000746F70205265672E207570646174657316
:10B56000293A2032392020202020202020200A00C3
:10B570005374617274204144493120436F6E766583
:10B580007273696F6E28436F6E74696E756F757331
:10B59000293A203520202020202020202020202073
:10B5A000202020202020202020202020207C554EDC
:10B5B000534E415028526573756D65205265672E54
:10B5C0002075706461746573293A2033302020201F
:10B5D00020200A0053746172742041444932204390
:10B5E0006F6E76657273696F6E28436F6E74696EE5
:10B5F000756F7573293A20362020202020202020C6
:10B60000202020202020202020202020202020203A
:10B61000207C5365742052657365742047504F2019
:10B6200050696E733A2033312020202020202020C2
:10B630002020202020200A0053746172742041448D
:10B64000493120526564756E64616E7420436F6E7B
:10B6500076657273696F6E2853696E676C652053E7
:10B66000686F74293A2037202020202020202020B5
:10B6700020202020207C4750494F205350492057FC
:10B680007269746520746F20536C6176653A20335B
:10B69000322020202020202020200A0053746172B4
:10B6A00074204144493120526564756E64616E7442
:10B6B00020436F6E76657273696F6E28436F6E7488
:10B6C000696E756F7573293A20382020202020205C
:10B6D0002020202020202020207C4750494F20532C
:10B6E000504920526561642066726F6D20536C6111
:10B6F00076653A20333320202020202020200A00A5
:10B70000526561642043522C205642415420262029
:10B7100049564241542052656769737465727328B3
:10B7200053696E676C652053686F74293A2039201D
:10B73000202020202020202020202020207C475056
:10B74000494F2049324320577269746520746F2035
:10B75000536C6176653A203334202020202020204D
:10B7600020200A00526561642043522C2056424139
:10B77000542026204956424154205265676973740B
:10B7800065727328436F6E74696E756F7573293AAD
:10B790002031302020202020202020202020202088
:10B7A000207C4750494F2049324320526561642034
:10B7B00066726F6D20536C6176653A2033352020B8
:10B7C0002020202020200A0052656164204F7665E9
:10B7D0007263757272656E742041444320526567CE
:10B7E00069737465722853696E676C652053686F5E
:10B7F00074293A20313120202020202020202020B0
:10B8000020202020207C20202020202020202020DC
:10B810002020202020202020202020202020202028
:10B82000202020202020202020200A005265616452
:10B83000204F76657263757272656E742041444361
:10B8400020526567697374657228436F6E74696E00
:10B85000756F7573293A2031322020202020202056
:10B860002020202020202020207C2020202020207C
:10B8700020202020202020202020202020202020C8
:10B8800020202020202020202020202020200A00EE
:10B890005265616420417665726167652043522C70
:10B8A0002056424154202620495642415420526598
:10B8B000676973746572732853696E676C6520538A
:10B8C000686F74293A20313320202020207C2020EA
:10B8D0002020202020202020202020202020202068
:10B8E0002020202020202020202020202020202058
:10B8F00020200A00526561642041766572616765A7
:10B900002043522C20564241542026204956424181
:10B91000542052656769737465727328436F6E743F
:10B92000696E756F7573293A2031342020202020EC
:10B93000207C2020202020202020202020202020AB
:10B9400020202020202020202020202020202020F7
:10B950002020202020200A005265616420416C6C68
:10B9600020435220616E64205642415420566F6C31
:10B9700074616765205265676973746572732853D3
:10B98000696E676C652053686F74293A20313520E1
:10B9900020202020207C202020202020202020204B
:10B9A0002020202020202020202020202020202097
:10B9B000202020202020202020200A0052656164C1
:10B9C00020416C6C20435220616E642056424154E9
:10B9D00020566F6C74616765205265676973746582
:10B9E000727328436F6E74696E756F7573293A2090
:10B9F0003136202020202020207C202020202020C4
:10BA00002020202020202020202020202020202036
:10BA100020202020202020202020202020200A005C
:10BA200053746172742041445620416C6C20436809
:10BA3000616E6E656C20436F6E76657273696F6EB2
:10BA40003A203137202020202020202020202020B4
:10BA5000202020202020202020202020207C20208A
:10BA600020202020202020202020202020202020D6
:10BA700020202020202020202020202020202020C6
:10BA800020200A005265616420416C6C20565220CF
:10BA90005265676973746572732852445620636FE8
:10BAA0006D6D616E6473293A20313820202020208A
:10BAB0002020202020202020202020202020202086
:10BAC000207C20202020202020202020202020201A
:10BAD0002020202020202020202020202020202066
:10BAE0002020202020200A005265616420416C6CD7
:10BAF00020525652205265676973746572732852DA
:10BB000044525641202620524452564220636F6DC3
:10BB10006D616E6473293A20313920202020202065
:10BB200020202020207C20202020202020202020B9
:10BB30002020202020202020202020202020202005
:10BB4000202020202020202020200A00526561642F
:10BB500020416C6C205652202620525652205265AD
:10BB600067697374657273285244562C205244528C
:10BB70005641202620524452564220636F6D6D611B
:10BB80006E6473293A203230207C2020202020202F
:10BB900020202020202020202020202020202020A5
:10BBA00020202020202020202020202020200A00CB
:10BBB0005265616420566F6C7461676520526567D9
:10BBC0006973746572732852444155584320262086
:10BBD00052444155584420636F6D6D616E64732902
:10BBE000284E41293A20323120202020207C20205C
:10BBF0002020202020202020202020202020202045
:10BC00002020202020202020202020202020202034
:10BC100020200A0053746172742041444155582019
:10BC2000416C6C204368616E6E656C20436F6E766C
:10BC3000657273696F6E3A203232202020202020F6
:10BC400020202020202020202020202020202020F4
:10BC5000207C202020202020202020202020202088
:10BC600020202020202020202020202020202020D4
:10BC70002020202020200A00526561642041444198
:10BC80005558204D6561737572656D656E743A2007
:10BC9000323320202020202020202020202020207F
:10BCA0002020202020202020202020202020202094
:10BCB00020202020207C2020202020202020202028
:10BCC0002020202020202020202020202020202074
:10BCD000202020202020202020200A00526561649E
:10BCE00020537461747573204320526567697374BF
:10BCF00065723A203234202020202020202020206D
:10BD00002020202020202020202020202020202033
:10BD10002020202020202020207C202020202020C7
:10BD20002020202020202020202020202020202013
:10BD300020202020202020202020202020200A0039
:10BD40005265616420416C6C20537461747573207A
:10BD50005265676973746572733A2032352020200A
:10BD600020202020202020202020202020202020D3
:10BD7000202020202020202020202020207C202067
:10BD800020202020202020202020202020202020B3
:10BD900020202020202020202020202020202020A3
:10BDA00020200A00000099C5ABCE320BCFD8561D1B
:10BDB0006416FDD307F49E31AC3A35FFC82C51E927
:10BDC00063E2FA2797AD0E683C63A5A65875C1B02B
:10BDD000F3BB6A7E9059099C3B97A2525F81C6448F
:10BDE000F44F6D8A2E5BB79E85951C50E183784693
:10BDF0004A4DD38829AFB06A82611BA4E6777FB22F
:10BE00004DB9D47CB9F6203312388BFD762EEFEB8A
:10BE1000DDE04425BE0227C715CC8C0971DAE81F86
:10BE2000DA1443D1C5F35C366E3DF7F80A2B93EE76
:10BE3000A1E53820C2075BC269C9F00C0DDF941A76
:10BE4000A6113FD4525ECB9BF99060559D8604436A
:10BE50003648AF8D55AACC6FFE6467A19A7203B7BE
:10BE600031BCA879EBA8726D4066D9A32470BDB52A
:10BE70008FBE167BEC5C75994792DE572384BA41DE
:10BE8000884A118F7C05E5C0D7CB4E0EB3DD2A184A
:10BE9000181381D67BF1E234D03F49FAB4292DEC56
:10BEA0001FE7862213A28A67B86C21A9DC7A45BFF6
:10BEB00077B4EE7114568D93BF98265DDB8E424B9E
:10BEC0007040E985840F1DCA2FC1B6044BD7D2122A
:10BED000E01979DC83FB1A3E2835B1F04C23D5E616
:10BEE000E7ED7E283DF9A43C96370FF2F2216BE492
:10BEF00059EFC02A3A0DA3C891C30806F5D56C10B6
:10BF00005E1BC7DEAA543391019A985F658CFC4989
:10BF1000CE425787ADA03465066E9FAB6278FBBDFD
:10BF2000C9B65073D6514F947D9FE45A1989804CFD
:10BF3000B2472B82D1A548607A6BE3AE1E7D87B8ED
:10BF4000B5B32C7641FCD839EA3273F78E2417E169
:10BF500025EABC2F4608DFCDEDC6740389D0101545
:10BF6000221EBBDBF80A61CF53C4CA0137D2AE1719
:10BF70009C1C05D9FFFE663B5430CDF53026A9E365
:10BF80009BE8022D6FA7F662C4695DACA07F39BA49
:10BF90000BB192746853F196C39D5A58A78B3E4ECD
:10BFA0000C4595802DE9F04107468846387810F019
:10BFB000030F16461D4633D03846FFF747F978BBC6
:10BFC000B8F1000F1CBFD8E900018619012D2ED150
:10BFD0003888C10415D5396A07F14402384600F0A3
:10BFE0004DF83A6B044602B93A69F968384600F0F0
:10BFF00045F8361B341A7A69F968384600F03EF87D
:10C00000261A1EB94DB916F1010F09D097F9030090
:10C010002A46314600F038F8064616F1010F09D1DC
:10C020002320AFF300804FF0FF30BDE8F081022DF8
:10C03000E8D1EBE7388810F4405F0ED07868F860FC
:10C0400038617861B86107F144017868F861396254
:10C0500007F13000002178623963B8F1000F05D094
:10C06000D8E9020107F13402C2E900013B884CF62D
:10C07000FF6003403B800020BDE8F081914234BF67
:10C08000511A0021084670473EB504000D00012AF0
:10C0900002D1FFF761F907E0022A07D100940020DE
:10C0A000019069460C20ABBE2D1801E0002A0CD18E
:10C0B0000094019569460A20ABBE002805D10022F4
:10C0C00021002800FFF725F901E00020C04303B05C
:10C0D00030BD10B50446E0682169884252D32188FA
:10C0E000C80547D44AF2010000EA0102012A07D03C
:10C0F00008044CBF4FF400704FF4844001432EE01D
:10C1000011F4406F02BF606804F14401884215D108
:10C110004FF40070F4F792F828B904F1440060601D
:10C12000401CA0600AE0218841F04001218060604D
:10C13000606100F500726068A260E0616068E060C4
:10C140002061A0616168A26894F90300521A00F0AE
:10C150001BF8218810F1010F05D141F484412180A1
:10C160004FF0FF3010BD38B94EF6FF70014041F47A
:10C1700082412180002010BD41F4A041218021692D
:10C1800008442061012010BD78B583B004000D0083
:10C190001600002C03D1F5F72FFB009000E000946F
:10C1A0000195029669460620ABBE01222100301A95
:10C1B000FFF7AFF804B070BD10B50446E068A169A0
:10C1C000884251D3218849F202030B40022B08D048
:10C1D00008044CBF4FF400704FF4844001432180A9
:10C1E0003BE001F4C042B2F5C04F06D1A1688842DD
:10C1F00003D32046FFF72AF878BB208810F4406F5D
:10C2000002BF606804F14401884217D14FF4007006
:10C21000F4F714F830B904F144006060E060401CA9
:10C22000A0600BE0218841F040012180E060606067
:10C23000606100F500726068A260E0616068A168FA
:10C240002061A161207841070AD502220021204601
:10C2500000F00CF810F1010F02D14FF0FF3010BDCB
:10C26000208840F4C0402080002010BD70B50446F6
:10C270000D461646AFF3008033462A46002120467D
:10C28000FFF790FE05462046AFF30080284670BDBC
:10C29000F0B40246106895681318506803EB500418
:10C2A000C0071CD54D441AE013F8017B05F8017B4B
:10C2B000491EF9D198B113F8011BC6F38106032E6C
:10C2C00008BF13F8016B01EB06214942801C294489
:10C2D00005D011F8016B05F8016B401EF9D1A3429E
:10C2E0000ED013F8016B16F0030104BF13F8011B05
:10C2F000C91C30090F28DBD113F8010B0F30D7E729
:10C30000F0BC02F10C00704738B50446AFF3008072
:10C310002088410409D5206A04F14401884204D2EE
:10C32000421C226212F8015D15E0206B10B1206101
:10C3300000202063E0682169884208D32046FFF787
:10C34000C8FE0128B8BF4FF0FF3504DBE068401C91
:10C35000E06010F8015D2046AFF30080284632BD52
:10C3600070B504460D462846AFF3008014F1010F66
:10C370001EBF2A6A05F143018A4206D02B884AF281
:10C38000010000EA0306012E02D04FF0FF340EE058
:10C390004FF6FF610B4043F4A0432B80286B18B984
:10C3A0002869696828632961501E2862047028463C
:10C3B000AFF30080204670BD38B50C46C5B22046AC
:10C3C000AFF30080E068A169884204D32046FFF7FC
:10C3D000F3FE00280FD4E068401CE06000F8015D27
:10C3E0002088010503D440050BD50A2D09D120462C
:10C3F000FEF72CFF28B12046AFF300804FF0FF304E
:10C4000032BD2046AFF30080284632BD49435B254C
:10C41000645D3A2053656C6563742047504F20502B
:10C42000696E20447269766520746F204869676878
:10C430000A00000049435B25645D3A2053656C6542
:10C4400063742047504F2050696E204472697665AE
:10C4500020746F204C6F770A000000000000412913
:10C46000211C191716151413121211111110101086
:10C470000F0F0F0F0E0E0E0E0E0E0E0D0D0D0D0DDD
:10C480000D000000303132333435363738396162CF
:10C49000636465666768696A6B6C6D6E6F707172F4
:10C4A000737475767778797A000000007363616E33
:10C4B000665F733A2062616420256C632C20256CD2
:10C4C000732C206F7220256C5B20617267756D651F
:10C4D0006E7400007363616E665F733A206261641C
:10C4E0002025632C2025732C206F7220255B206172
:10C4F0007267756D656E74000448054A016841F401
:10C50000700101604FF000601060704788ED00E03E
:10C5100008ED00E00000000000000000010203043C
:10C520000607080900000000000000000000244089
:10C530000000000000005940000000000088C340D7
:10C540000000000084D797410080E03779C3414361
:10C55000176E05B5B5B89346F5F93FE9034F384D69
:10C56000321D30F94877825A3CBF737FDD4F157515
:10C570007047FEE7FEE7FEE7FEE77047704770474B
:10C58000704700F017B88020FCF7BDB80548FCF7ED
:10C59000EABC0548FCF74BBB0448FDF706BE04485F
:10C5A000FDF703BED808002088030020E004002027
:10C5B0002005002010B5054C2068C10304D500F00B
:10C5C00007F84FF48030206010BD0000143C01409B
:10C5D000704700004661696C656420746F20616C6F
:10C5E0006C6F636174652077726974655F627566EC
:10C5F000666572206172726179206D656D6F727906
:10C60000000000004750494F2049324320577269CB
:10C610007465206461746120746F20536C61766569
:10C6200020636F6D706C6574656400004750494FFE
:10C630002049324320526561642064617461206640
:10C64000726F6D20536C61766520636F6D706C65E1
:10C65000746564004661696C656420746F20616C68
:10C660006C6F6361746520706172736520726564BC
:10C670007672206D656D6F72790000004661696C9D
:10C68000656420746F20616C6C6F636174652073E6
:10C69000706920726561642064617461206D656DEC
:10C6A0006F7279007363616E665F733A20626164D2
:10C6B00020666C6F6174696E672D706F696E74208F
:10C6C000617267756D656E740000000010B50749F2
:10C6D00079441831064C7C44163404E00A68081D7D
:10C6E000114488470146A142F8D110BD0401000061
:10C6F000200100004164693120726564756E6461D7
:10C700006E7420636F6E76657273696F6E20636FEF
:10C710006D706C65746564004750494F20535049F3
:10C7200020577269746520746F20536C61766520A0
:10C73000436F6D706C657465640000004750494F2D
:10C740002053504920526561642066726F6D2053FA
:10C750006C61766520436F6D706C65746564000074
:10C760004661696C656420746F20616C6C6F6361F5
:10C770007465207061727365207672206D656D6FCF
:10C78000727900004661696C656420746F20616C89
:10C790006C6F6361746520636D642061727261798E
:10C7A000206D656D6F727900506C656173652065F1
:10C7B0006E746572206C6F6F70206D656173757239
:10C7C0006D656E7420636F756E743A004EF6885115
:10C7D000CEF20001086840F470000860BFF34F8F8C
:10C7E000BFF36F8F4FF00070E1EE100A704700004A
:10C7F000CF4EFFFF040600004003002000000000B1
:10C8000091FAFFFF00020000F2010000000000208A
:10C8100000F00DF8002801D0FFF758FFAFF30080BB
:10C820000020AFF30080FDF775F8FCF711FE012042
:10C83000704700000548014603B4684680F3098844
:10C84000AFF30080FFF7C2FFFFF7E2FFA5EDF5FEB3
:10C8500038B504460D46284600F006F8A84218BF31
:10C860000024204632BD00000149FFF7A5BD00BFEE
:10C87000480200200148804701480047F9C40008E9
:10C8800035C800080248FFF73FBD0149FFF768BD02
:10C89000000200200846002A18BFFFF7F3BFFFF789
:10C8A000F4BF00000000000001020304FFF7FEBF18
:10C8B000FFF7FEBFFFF7FEBFFFF7FEBFFFF7FEBFAC
:10C8C000FFF7FEBFFFF7FEBFFFF7FEBFFFF7FEBF9C
:10C8D000FFF7FEBFFFF7FEBFFFF7FEBFFFF7FEBF8C
:10C8E000FFF7FEBFFFF7FEBFFFF7FEBFFFF7FEBF7C
:10C8F000FFF7FEBFFFF7FEBFFFF7FEBFFFF7FEBF6C
:10C90000FFF7FEBFFFF7FEBFFFF7FEBFFFF7FEBF5B
:10C91000FFF7FEBFFFF7FEBFFFF7FEBFFFF7FEBF4B
:10C92000FFF7FEBFFFF7FEBFFFF7FEBFFFF7FEBF3B
:10C93000FFF7FEBFFFF7FEBFFFF7FEBFFFF7FEBF2B
:10C94000FFF7FEBFFFF7FEBFFFF7FEBFFFF7FEBF1B
:10C95000FFF7FEBFFFF7FEBFFFF7FEBFFFF7FEBF0B
:10C96000FFF7FEBFFFF7FEBFFFF7FEBFFFF7FEBFFB
:10C97000FFF7FEBFFFF7FEBFFFF7FEBFFFF7FEBFEB
:10C98000FFF7FEBFFFF7FEBFFFF7FEBFFFF7FEBFDB
:10C99000FFF7FEBFFFF7FEBFFFF7FEBFFFF7FEBFCB
:10C9A000FFF7FEBFFFF7FEBFFFF7FEBFFFF7FEBFBB
:10C9B000FFF7FEBFFFF7FEBFFFF7FEBFFFF7FEBFAB
:10C9C000FFF7FEBFFFF7FEBFFFF7FEBFFFF7FEBF9B
:10C9D000FFF7FEBFFFF7FEBFFFF7FEBFFFF7FEBF8B
:10C9E000FFF7FEBFFFF7FEBFFFF7FEBFFFF7FEBF7B
:10C9F000FFF7FEBFFFF7FEBFFFF7FEBFFFF7FEBF6B
:10CA0000FFF7FEBF90030723B9E40001120A0DF3FC
:10CA1000FF010001F1310164068803002060050078
:10CA2000205C221008F0050724F400F62F0008040B
:10CA300052FF01E3CA171420040000522E00084CD4
:10CA40002002800100204B2002DB5400080852D550
:10CA50000812F10812D90443055510210112454866
:10CA6000123D04432B173C21011007010400004430
:10CA70000200204504524404211BA10852300CF14D
:10CA80000B0110070204010188080020D804528815
:10CA90000421346108128C44F213784850020802D1
:10CAA0000238405238042134610812D444F212C0D2
:10CAB00048120024124804F206902C655C19ED120D
:10CAC000242C140326000400062A002F0A00090063
:10CAD0000B0044004600480007000D00030005005D
:10CAE00030003100320033003407180721072200DC
:0DCAF0002C002E002D002F0027001B001F22
:040000050800C835F2
:00000001FF
